:020000020000FC
:100000000C94E2110C94840D0C94990D0C94CA116B
:100010000C94800D0C94810D0C94820D0C94830D26
:100020000C946D0D0C946E0D0C946F0D0C94700D62
:100030000C94710D0C94720D0C94730D0C94740D42
:100040000C94750D0C94760D0C94AE0D0C947A0DE9
:100050000C9487100C94CC100C947B0D0C94780DA0
:100060000C94EF100C94770D0C94790D0C947F0D7B
:100070000C947C0D0C947D0D0C947E0D8954400BDA
:10008000B83630303000895A1C05783238303000AC
:10009000895A1C04B03234303000895A1C041A3298
:1000A00031303000895A1C03843138303000895790
:1000B0002E01F4313030300089572E00C820343002
:1000C000300089572E007D20323530001F28641102
:1000D0000001B0001D00B8000D001F2864110001D0
:1000E000B8000D00E0000D001F2864110001E000C1
:1000F0000D00E8001D001F2864110001BB001D0059
:10010000C3000D001F2864110001C3000D00D500BD
:100110000D001F2864110001D5000D00DD001D0039
:100120001F2864110001BC001D00C4000D001F2821
:1001300064110001C4000D00D4000D001F286411DB
:100140000001D4000D00DC001D001F286411000117
:10015000BD001D00C5000D001F2864110001C50071
:100160000D00D3000D001F2864110001D3000D0005
:10017000DB001D001F2864110001BE001D00C60029
:100180000D001F2864110001C6000D00D2000D00F3
:100190001F2864110001D2000D00DA001D001F2885
:1001A00064110001C0001D00C8000D001F2864116B
:1001B0000001C8000D00D0000D001F2864110001CF
:1001C000D0000D00D8001D001F2864110001C200DE
:1001D0001D00CA000D001F2864110001CA000D0097
:1001E000CE000D001F2864110001CE000D00D600C6
:1001F0001D001F2864110001C4001D00CB000D006C
:100200001F2864110001CB000D00CD000D001F2838
:1002100064110001CD000D00D5001D0006F1582726
:10022000102032304B0006F1580B54353830300076
:1002300006F1580578323830300006F1580514328E
:100240003630300006F158041A323130300006F1F1
:100250005803E8323030300006F15803843138302A
:10026000300006F15801F4313030300006F158000A
:10027000FA203530300006F15800C8203430300004
:1002800006F1580096203330300006F158007D20EA
:100290003235300006F158003E20313235001F283B
:1002A00064110001B0001D00B70010001F28641188
:1002B0000001B7001000E10010001F2864110001C8
:1002C000E1001000E8001D001F2864110001B200C9
:1002D0001D00B90010001F2864110001B9001000B2
:1002E000DF0010001F2864110001DF001000E6008D
:1002F0001D001F2864110001BC001D00C300100078
:100300001F2864110001C3001000D50010001F2831
:1003100064110001D5001000DC001D001F286411CD
:100320000001BD001D00C40010001F286411000161
:10033000C4001000D40010001F2864110001D40074
:100340001000DB001D001F2864110001BE001D000D
:10035000C50010001F2864110001C5001000D30063
:1003600010001F2864110001D3001000DA001D00E6
:100370001F2864110001BF001D00C60010001F28C7
:1003800064110001C6001000D20010001F28641183
:100390000001D2001000D9001D001F2864110001C7
:1003A000C0001D00C70010001F2864110001C70015
:1003B0001000D10010001F2864110001D1001000AE
:1003C000D8001D001F2864110001C1001D00C800D5
:1003D00010001F2864110001C8001000D000100098
:1003E0001F2864110001D0001000D7001D001F2835
:1003F00064110001C2001D00C90010001F28641113
:100400000001C9001000CF0010001F286411000176
:10041000CF001000D6001D001F2864110001C3008A
:100420001D00CA0010001F2864110001CA0010003E
:10043000CE0010001F2864110001CE001000D5006E
:100440001D001F2864110001C4001D00CB00100016
:100450001F2864110001CB001000CD0010001F28E0
:1004600064110001CD001000D4001D001F2864118C
:100470000001C5001D00CC0010001F286411000100
:10048000CC001000CC0010001F2864110001CC002B
:100490001000D3001D001F2864110001C6001D00BC
:1004A000CD0010001F2864110001CD001000CB000A
:1004B00010001F2864110001CB001000D2001D00A5
:1004C0001F2864110001CC002000CC000A001F2866
:1004D0006411020098000A00FF001D001F24BE00E6
:1004E00000001F2867010120504120566F6C747373
:1004F0002D3E20524620436F6D702D3E202020203F
:1005000020414C432D3E20202020205357522D3E89
:1005100020467764205077722D3E5265666C2050DD
:1005200077722D3E20504120437572722D3E4476E5
:100530007220437572722D3E0C1F286701011F2423
:10054000780002001F286701026B487A1F5800FFDD
:100550001F5811FF1F5812FF1F5813FF1F5814FF79
:100560001F5815FF1F5816FF1F5817FF1F5818FF59
:100570000B1F2867010400000000001F286701020C
:100580000A2E000000FF0B1F2867010420202020F6
:1005900020000B1F286701040000001F28670102CC
:1005A0001F24380002000000002E000000FF1F245E
:1005B000000005001F2867010154783A0000000080
:1005C000002E00001F286411020098000800FF00A0
:1005D0002E001F24420005001F28670101523AFF28
:1005E00043572855534229204357284C534229202A
:1005F00055534220202020204C53422020202020F0
:10060000414D202020202020464D20202020202049
:100610004449472855534229444947284C534229C5
:100620001F24000005001F28670101583AFF1F24FE
:10063000DA0007001F28670101502DFF1F24CC009E
:1006400007001F286701015420FF1F2482000500B6
:100650001F28670101FF1F249A0004001F2867015B
:10066000012A393A20202020202020343AFF1F245C
:100670008E0000001F286701014C6F636BFF1F2471
:10068000000002001F286701024F7574206F66206A
:1006900062616E6421FF1F24000002001F286701B1
:1006A0000252414D207465737420706173736564E8
:1006B0006661696C65640C1F24000002001F2867D6
:1006C000010250726F632073796E63206661696CFA
:1006D00065641F24880001001F2867010120206134
:1006E00041624263436444654566466747684869BA
:1006F000496A4A6B4B6C4C6D4D6E4E6F4F7050712A
:100700005172527353745475557656775778587999
:10071000597A5A303132333435363738393F2C2E06
:100720002F2D3D2B282623252A3A3B2140292427FB
:100730005F3C1F24000004001F28670101202020C7
:10074000202020202020202020FF0C1F2420000219
:10075000001F2867010441434E3641477A3641481D
:100760009336414CAC36414EC63641501937415252
:10077000F03641543337425253374341A73743424F
:10078000953743467837434CDC374352ED37435374
:10079000FE37435467374355CB3743581A384446DE
:1007A0003238444E2B384454433844565D38455310
:1007B0007138464194384642A0384644AC384649E0
:1007C000C838464EF038465270394653AD39465413
:1007D0008C394657CA3946585A3A4659823A47548C
:1007E000A63A4853CF3A4944E53A4946ED3A495288
:1007F000193949536A3B49582B3949593B394B4DB3
:10080000D33B4B53F43B4B59143C4C433F3C4C4B78
:10081000583C4C54733C4D428C3C4D43A53C4D449C
:10082000CC3C4D47013D4D521A3D4D576C3D4E421B
:10083000A63D4E54C23D4E57DB3D5041FD3D504319
:10084000293E50446D3E504C8D3E504DAA3E505274
:10085000C93E5053ED3E5054063F5057403F524121
:100860005E3F52438A3F52448F3F5246B53F524704
:10087000C83F524BE53F524D0D40525055405254E7
:100880005B4052559C3F52587F40534290405343E7
:10089000C74053446541534596415349DE40534D4B
:1008A000AD415350F5405351C94153531641535430
:1008B000374153564E415443E64154460542544C49
:1008C0001642544D2F4254523E425458AF40555058
:1008D0008D3856415B42564474425647A54256589D
:1008E000B7425843074358440C435854E3425855C1
:1008F0001943585632431F24580000000808435734
:100900002855534229204357284C534229205553F8
:100910004220202020204C53422020202020414DE6
:10092000202020202020464D202020202020444927
:10093000472855534229444947284C5342291F24EC
:100940000000070000044147432D04044175746F03
:1009500046617374536C6F774F6666201F243C00AA
:10096000070000034E422D02046F6666206F6E2062
:1009700020FF1F246C0007000404505454205054DE
:100980005443564F5820564F58431F248A0007009F
:10099000000352782D02015452FF1F24AC000700BF
:1009A000000354782D02014142FF1F2498000100EA
:1009B00000074D657465723A20080A504120566F51
:1009C0006C74732020524620436F6D7020202041AC
:1009D0004C4320202020202020535752202020202C
:1009E00020202046776420507772202020526566B0
:1009F0006C20507772202050412043757272202065
:100A00002044767220437572722020FF1F249800C4
:100A10000200000D4272696768746E6573733A2054
:100A20002008044C6F77304C6F77314C6F77324C25
:100A30006F77334D6564314D6564324D656433487D
:100A4000696768FF1F2498000300000750205320A7
:100A5000423A20020A4F6666202020202020204FA4
:100A60006E2020202020202020FF1F24980004003A
:100A7000000F44697370207265732028487A293A00
:100A800020020231302031FF1F24980005000007AA
:100A90004E422050573A20030A53686F7274202048
:100AA0002020204D656469756D202020204C6F6EDC
:100AB00067202020202020FF1F2498000100000E26
:100AC0005054542D524620286D73293A20201E037D
:100AD00020203120203220203320203420203520B7
:100AE0002036202037202038202039203130203176
:100AF000312031322031332031342031352031362C
:100B00002031372031382031392032302032312025
:100B10003232203233203234203235203236203205
:100B2000372032382032392033301F249800020019
:100B3000000A504320417564696F3A2002074469F6
:100B40007361626C65456E61626C65201F2498005C
:100B50000300000A547820417564696F3A20020747
:100B60004D6963202020204C696E652020201F24C1
:100B700098000400000C4C6F636B2074696D657203
:100B80003A2004054F666620203130732020333030
:100B900073202036307320201F2498000500000C9D
:100BA000506F77657220736176653A2004054F6651
:100BB00066202031356D696E33306D696E36306D6B
:100BC000696E1F2498000100000C5069746368204E
:100BD00028487A293A2001F81F2498000200000DC5
:100BE0005370656564202877706D293A2001F8FFFD
:100BF0001F2498000300000E456E68616E636564F3
:100C0000205353423A2002034F6666204F6E1F2442
:100C100098000400000E464D2044657620286B485D
:100C20007A293A200303322E30342E30352E30FF0D
:100C30001F2498000500000F4C6963656E736520E2
:100C4000636C6173733A20050245204120472054AC
:100C5000204E20FF1F24980001000009565041201B
:100C60002856293A2001FAFF1F24980002000009A3
:100C7000495041202841293A2001FAFF1F249800B9
:100C800003000009494476202841293A2001FAFF4F
:100C90001F24980004000009436D70286442293A1B
:100CA0002001FAFF1F24980005000009414C432051
:100CB0002856293A2001FAFF1F2498000100000954
:100CC000535752202020203A2001FAFF1F24980079
:100CD00002000009467764202857293A2001FAFFCC
:100CE0001F24980003000009526566202857293AFE
:100CF0002001FAFF1F2498000400000A2020202071
:100D0000202020202020020720202020202020201A
:100D10002020202020201F2498000500000A2020E9
:100D200020202020202020200207202020202020FA
:100D300020202020202020201F2498000100000EC9
:100D4000564F58206761696E3A2020202020FFF816
:100D50001F2498000200000E564F582073656E73D2
:100D60003A2020202020FFF81F2498000300000EC6
:100D7000416E7469564F58206761696E3A20FFF8DA
:100D80001F2498000400000E564F5820646C7928E8
:100D900031306D73293AFFF81F2498000500000ACE
:100DA0004D696320426961733A2002074F666620ED
:100DB0002020203920566F6C74731F249800010086
:100DC0000005416D703A20040C4E6F6E65202020A6
:100DD0002020202020496E742031305720202020F0
:100DE00020496E74203130305720202020496E7405
:100DF00020313030572B457874FF1F2498000200B3
:100E0000000C4B65796572204D6F64653A200305CF
:100E100049616D624149616D6242556C74696DFF53
:100E20001F2498000300000E4661726E73776F7284
:100E300074683A20202011034F6666202035202058
:100E40003620203720203820203920313020313101
:100E500020313220313320313420313520313620D9
:100E60003137203138203139203230FF1F249800AB
:100E70000400000E53424920646C792831306D73B0
:100E8000293AFFF81F2498000500000E4642492029
:100E9000646C79286D73293A2020FFF81F2498008C
:100EA0000100000E58766572746572204672657195
:100EB0003A2017036F6666353020353220353420EE
:100EC00031343431343632323232323434323034F6
:100ED00032323432343432363432383433303433DC
:100EE00032343334343336343338343430343432C7
:100EF000343434343436343438FF1F24980002003C
:100F000000094454523D5054543A2002084E6F2078
:100F100020202020205965732020202020FF1F241E
:100F200098000300000B4261756420726174653A99
:100F3000200506202039363030203139323030203B
:100F40003338343030203537363030313135323087
:100F500030FF1F2498000400000A48616E64736823
:100F6000616B653A02072020204E6F6E6543545333
:100F70002F5254531F2498000500000D5475726EB3
:100F80006F6E20646973703A200204204F66664DCC
:100F9000736731FF1F2498000100000B5363616EDB
:100FA00020747269703A20050620202020533520D5
:100FB000202020533620202020533720202020536B
:100FC00038202020205339FF1F2498000200000CF5
:100FD0005363616E2073746172743A20FFF81F24AA
:100FE00098000300000B5363616E2073746F703AB6
:100FF00020FFF8FF1F2498000400000E4672657160
:1010000020696E6328487A293A20090363686E20B4
:10101000313031303020314B31304B31354B323083
:101020004B32354B35304BFF1F2498000500000D27
:101030004477656C6C20286D73293A2020050420C4
:1010400031303020323530203530303130303035AD
:10105000303030FF1F24980001000006526F6F6689
:101060003A20020B37302E3030304D487A2020376E
:10107000302E3435354D487A20201F249800020048
:101080000008394D487A2D313A2001093630303088
:101090002020202020FF1F24980003000008394D45
:1010A000487A2D323A20090936303030202020206D
:1010B00020323830302020202020323430302020A0
:1010C0002020203231303020202020203138303094
:1010D00020202020203130303020202020203430AB
:1010E00030202020202020323530202020202020B9
:1010F0006E6F6E652020202020FF1F2498000400C2
:101100000008394D487A2D333A20090936303030FD
:10111000202020202032383030202020202032345F
:10112000303020202020203231303020202020205C
:101130003138303020202020203130303020202025
:101140002020343030202020202020323530202034
:10115000202020206E6F6E652020202020FF1F247D
:10116000980005000008394D487A2D343A200909C5
:1011700036303030202020202032383030202020DF
:1011800020203234303020202020203231303020D6
:1011900020202020313830302020202020313030D5
:1011A00030202020202034303020202020202032E9
:1011B00035302020202020206E6F6E6520202020DA
:1011C00020FF1F2498000100000A3435354B487A6F
:1011D0002D313A20020732304B2020202035383084
:1011E000302020201F2498000200000A3435354B9F
:1011F000487A2D323A200E0732304B2020202035FD
:101200003830302020203238303020202032363024
:101210003020202032313030202020323030302039
:101220002020313830302020203130303020202034
:101230003530302020202034303020202020333022
:10124000302020202032353020202020313235201F
:101250002020206E6F6E652020201F249800030040
:10126000000A3435354B487A2D333A200E07323098
:101270004B202020203538303020202032383030AC
:1012800020202032363030202020323130302020D3
:1012900020323030302020203138303020202031B2
:1012A00030303020202035303020202020343030A5
:1012B00020202020333030202020203235302020C4
:1012C0002020313235202020206E6F6E65202020B6
:1012D0001F2498000400000A3435354B487A2D3419
:1012E0003A200E0732304B20202020353830302075
:1012F000202032383030202020323630302020205C
:10130000323130302020203230303020202031382F
:101310003030202020313030302020203530302037
:101320002020203430302020202033303020202056
:101330002032353020202020313235202020206EF0
:101340006F6E652020201F2498000500000D467553
:101350006C6C204475706C65783A2002044F6666A8
:10136000204F6E2020FF1F249800010000095246E4
:10137000472063616C3A20FFF8FF1F2498000200A9
:10138000000C4147432043572F5353423A20FFF864
:101390001F2498000300000941474320414D3A2093
:1013A00020FFF8FF1F249800040000085478204113
:1013B0004C433A2002094F66662020202020204F0F
:1013C0006E202020202020201F2498000500000DE2
:1013D000547842572063616C205353423AFFF8FF20
:1013E0001F2498000100000C464D2F4946207465CB
:1013F00073743A2002054F666620204F6E2020202D
:101400001F2498000200000B532F50777220636155
:101410006C3A2002064F66662020204F6E20202066
:1014200020FF1F2498000300000D547820536866A5
:1014300028555342293A20FFF8FF1F249800040042
:10144000000D547820536866284C5342293A20FFF7
:10145000F8FF1F2498000500000D5443584F2054F6
:101460007765616B3A2020FFF8FF1F249800010088
:1014700000054D7367313A010CFF1F2498000200EC
:1014800000054D7367323A010CFF1F2498000300DA
:1014900000054D7367333A010CFF1F2498000400C8
:1014A00000054D7367343A010CFF1F2498000500B6
:1014B00000054D7367353A010CFF1F2498000100A9
:1014C00000054D7367363A010CFF1F249800020097
:1014D00000054D7367373A010CFF1F249800030085
:1014E00000054D7367383A010CFF1F249800040073
:1014F00000054D7367393A010CFF1F249800050061
:1015000000054D7331303A010CFF1F249800010093
:10151000000E436C722074756E6572206D656D3AB5
:101520000203204E6F5965731F24980002000008C3
:101530004320287046293A2001F81F249800030010
:10154000000E4320736964653A202020202020206B
:101550000203416E745478201F2498000400000890
:101560004C20286E48293A2001F81F2498000500D5
:10157000000E466F72636520726574756E653A2061
:1015800002034E6F205965731F249800010000105C
:10159000507263312052657620412E30312E323622
:1015A000010120FF1F2498000200000950726332DD
:1015B0002052657620FFF8FF1F2498000300000AE0
:1015C0002020202020202020202002072020202052
:1015D000202020202020202020201F2498000400EC
:1015E000000A202020202020202020200207202068
:1015F0002020202020202020202020201F24980090
:101600000500000E52652D70726F6772616D207556
:10161000503A0203204E6F5965731F248A00070059
:101620000004464470780000240033003E004A0065
:1016300052005A008B00A700BA00C9000000240025
:1016400033003E004A005200E1001A012B013C0128
:1016500051010000240033003E004A0052006601A0
:1016600071017D018C019D010000240033003E00CA
:101670004A005200AF01B901C301CD01D7010000FA
:10168000240033003E004A005200E101EB01F50165
:10169000FF0110020000240033003E004A00520007
:1016A00021022D02390245025102000024003300BC
:1016B0003E004A005200620282029502BB02C7024B
:1016C0000000240033003E004A005200D30202030F
:1016D00014032E033F030000240033003E004A00A1
:1016E00052004F03690374037F0399030000240031
:1016F00033003E004A005200AF03C203D00302048D
:1017000034040000240033003E004A005200660406
:101710007704B204ED0428050000240033003E00E5
:101720004A005200380542054D055705690500007D
:10173000240033003E004A005200750585059605D9
:10174000A205AE050000240033003E004A0052000E
:10175000BA05C205CA05D205DA0500002400330027
:101760003E004A005200E205EA05F205FA050206CB
:101770000000240033003E004A0052000A06190609
:10178000220631063A060000240033003E004A00DB
:10179000520049065706610672068306FF010707D5
:1017A000FA050303FA04010120000303FB0401010D
:1017B000FB0301011E04070738000707FB060101B0
:1017C0002E000101FA0203021D001F1D1E0001016F
:1017D000FB05010130000303300203031700FFFF84
:1017E0001900FFFF30070101360003021F00070444
:1017F0000B00FFFF0700FFFF0900FFFF0D00FFFFC9
:101800000F00FFFF0100FFFF0300FFFF0500FFFFC8
:1018100000000000000000001700FFFF1800FFFF9D
:101820001900FFFF1A00FFFF3A0701011E01030321
:101830001F04030228001F101B00FFFF1C00FFFFF6
:1018400031001F162F060101270007043700010190
:10185000280701012200070423007F5424007F543D
:1018600025000F08260007040E0001010F000F00DD
:1018700010000F0811000F0812000F0813000F01CD
:1018800014000F0D15000F0D16000F0D1F030101A1
:101890002B00FFFF2C00FFFF2D00FFFF3006010192
:1018A0003200FFFF30040101300501013300FFFF6A
:1018B0003400FFFF3500FFFF400000004100000042
:1018C000420000004300000044000000450000000A
:1018D00046000000470000004800000049000000EA
:1018E000290001011B00FFFF290101011D00FFFF6D
:1018F00029020101000000003900FFFF0000000084
:10190000000000002A00010132003400360090007F
:101910009200DE00E000A401A601A801AA01AC012A
:10192000AE01B001B201B401B601B801BA01BC0107
:10193000BE01C001001B77403E000102FFFF001EF8
:1019400084803C000102FFFF003567E03E00FFFF9E
:10195000FFFF0035C9883EFF010203040036EE8018
:101960003CFF01020304003875203EFF01FFFFFF2A
:101970000039FBC03EFFFF02FFFF003D09003C00B5
:101980000102FFFF005156443D000102FFFF0051DC
:1019900094C43D000102FFFF0051E2E43D0001025A
:1019A000FFFF0051F66C3D000102FFFF0052736C17
:1019B0003D000102FFFF006ACFC03E00FFFFFFFFB6
:1019C000006B31683EFF01020304006CB8083CFF65
:1019D000FF020304006D7B583EFFFF02FFFF006F14
:1019E00063A03C000102FFFF009A1D203E0001029F
:1019F000FFFF009AE0703C000102FFFF00D59F80CE
:101A00003E00FFFFFFFF00D601283EFF0102FFFF5F
:101A100000D7E9703CFF0102FFFF00D84B183EFFE2
:101A200001FFFFFF00D90E683EFFFF02FFFF00DA53
:101A3000F6B03C000102FFFF0113B2203E0001029C
:101A4000FFFF011538C03C000102FFFF01406F405D
:101A50003E00FFFFFFFF0140D0E83EFF010203040C
:101A600001437C803CFF010203040143DE283EFF6A
:101A700001FFFFFF0144A1783EFFFF02FFFF014786
:101A80004D103C000102FFFF017BCA903E000102A5
:101A9000FFFF017D51303C000102FFFF01AB3F0021
:101AA0003E000102FFFF01B2E0203CFFFFFF030404
:101AB00001C52FA03C000102FFFF0F37C0490F38BE
:101AC00030220F389FFB0F3830220F37C0490F37B5
:101AD00050700F36E0970F3750701895189518957D
:101AE000189518951895189518951895189518958E
:101AF000189518951895189518951895189518957E
:101B00001895189518951895FFB60F931F932F9356
:101B10000091D003002341F410E20E94F53311E05C
:101B200005FD1FEF1093D0032F911F910F91FFBE62
:101B30001895FFB60F931F932F930091CF030023A7
:101B400041F410E20E94F53311E004FD1FEF109301
:101B5000CF032F911F910F91FFBE1895FFB60F92E3
:101B60001F920F931F932F933F93AF93BF93CF93E6
:101B7000DF93EF93FF93B0911404A0911504109795
:101B800029F01197B0931404A0931504A0919E021C
:101B9000B0919D02109729F01197A0939E02B093E7
:101BA0009D020091A002002319F00A950093A00263
:101BB0000091CE0407FF0E948D3100915B0200234B
:101BC00061F00A9541F400915A02002331F0222479
:101BD0000E948D3102C000935B020091170407FF41
:101BE00017C010911804112399F406FD03C00027B3
:101BF000112707C0109119041A9532F410E2012739
:101C000014E62CE020931804109319040093170491
:101C100000911604002319F00A9500931604009110
:101C2000030400230AF069C0A091FA03B091F903FC
:101C30001197A093FA03B093F90309F05EC00091E5
:101C400001040093F903009102040093FA03009148
:101C5000D504002309F011C00091D1041091D404DF
:101C600003951395011711F40091D3040093D10447
:101C70000E944E350E94194440C010E00E94C634B4
:101C8000302F31702D911D910C91AF93BF93109017
:101C9000FB030090FC03000E111E00E0201F301F0C
:101CA00031703F932F931F920F9211E00E94C63420
:101CB000302F31702D911D910C910F900016002D39
:101CC0000F900106102D0F900206202D0F90030695
:101CD000302D49F044F03091FD032091FE03109126
:101CE000FF0300910004BF91AF910C931E932E93BC
:101CF0000E910E7F3170302B3C93B0910808A0916B
:101D000009081097B1F01197B0930808A09309083B
:101D100081F40FEF009327020093E1030093C903BE
:101D20000093510300938B020093640204E100933B
:101D30004701B0919F06A091A0061097C1F011979E
:101D4000B0939F06A093A00691F4F4E0E0EBAA27DD
:101D5000BB27D1E0C1EE0E943731102F008101175F
:101D600011F00E943E31119631962197A1F7B09162
:101D7000A106A091A206109761F01197B093A10659
:101D8000A093A20631F40FEF0093AC0201E00093A0
:101D90009303B091F503A091F603109749F01197C2
:101DA000B093F503A093F60319F401E00093F30355
:101DB00000915802023321F003950093580209C0A4
:101DC00000915A02002329F401E000935A020E9474
:101DD0008D313FEF00915302002359F00A95009393
:101DE0005302002399F410E20E94F5330093360168
:101DF0000DC010E20E94F53302FF05C003FF03C0CF
:101E00000093360103C002E30093530200919E0643
:101E1000002319F00A9500939E060091320110915B
:101E20003301011709F058C0009134010F7B109164
:101E300035011F7B011731F06624009134010074D5
:101E4000102BF8C000912902002319F00A95009385
:101E5000290200912D01002309F074C011270E946E
:101E6000F5331091A80210FD0F7710FD1095109317
:101E7000A80210915802113319F00F3F09F462C003
:101E80001091F30317FF11681093F30310913201BF
:101E900020E80090D00110909A010128109099013B
:101EA000012800FC006810FC006407FF122726953B
:101EB00006FF1227269505FF1227269504FF1227F5
:101EC000269503FF1227269502FF1227269501FF6C
:101ED0001227269500FF122700913201012706FFE5
:101EE00002C016FD3E7F3093080407FF0AC0009130
:101EF00034010C70C9F421E017FF2FEF2093CB01C0
:101F000013C004FF11C030910F040091110404307C
:101F10002CF414FD316014FF3E7F04C014FD3068C2
:101F200014FF3F7730930F04109332011093330165
:101F300010955090370110933701012F10E30E9444
:101F4000F533B6C010E10E94F533202F00741091D4
:101F500034011074102739F01FEF002309F411E049
:101F6000109313040AC010911304113034F0139528
:101F700017300CF0112710931304109134011F7BBC
:101F8000012B0093340100912D01002309F091C031
:101F9000022F0F7B3091080410FF03233FEF309393
:101FA00008041091A90210FD0B7F10FD10951093ED
:101FB000A9021091AA0210FD077F10FD1095109341
:101FC000AA0210919B0110FD0E7F10FD1095109339
:101FD0009B0110915802113319F00F3B09F46CC0AA
:101FE0001091F30317FF11681093F303109134015C
:101FF00020E866240090D00110909A01012809F091
:102000000C610090990100FC016007FF6094269527
:10201000269505FF1227269504FF1227269503FF14
:102020001227269502FF1227269501FF12272695D3
:1020300000FF122710933401109335011095509032
:102040003A0110933A01012F10E60E94F533662001
:1020500019F02FEF2093C3020091CE04087041F5D0
:1020600000913A010525087029F001E053FE0FEFB9
:102070000093C70100913A010525047029F001E0A1
:1020800052FE0FEF0093C90100913A01052502703D
:1020900079F051FE03C00E94122F07C00027009361
:1020A000A1060093A2060093AC020FEF00939303E6
:1020B00006E90A9500932D01009151020023B9F41D
:1020C00000913601007410915202102710E069F05F
:1020D00010E20E94F533202F00740093520211E0A9
:1020E000207C11F0203C09F41FEF1093510200EE08
:1020F00006BDFF91EF91DF91CF91BF91AF913F91DD
:102100002F911F910F911F900F90FFBE1895FFB652
:10211000AF93BF930F931F932F930091AB060023B0
:1021200019F00091C60031C0B6E0ADEA1091AC06DE
:102130000027A10FB01F0091C600003234F10C93AC
:1021400013952091E7042223A1F0163440F020914A
:10215000A50220FD0EC021682093A5020AC01A30F6
:1021600040F42091A50220FD04C02E772160209329
:10217000A502103511F01093AC060B3331F40FEFBC
:102180000093AB0600270093AC062F911F910F918F
:10219000BF91AF91FFBE1895FFB6AF93BF930F935A
:1021A0001F930091FD06002331F40091C1000F7DC3
:1021B0000093C1000EC0B6E0AFEF1091FE06101BF9
:1021C0000A950093FD060027A10FB01F0C91009304
:1021D000C6001F910F91BF91AF91FFBE1895FFB63A
:1021E0000F921F920F931F932F933F93AF93BF9321
:1021F0000091E004007161F10091340106FF28C0F4
:10220000EF93FF93FAE1EAEB11270091EB03000F44
:10221000111F000F111FE00FF11F05910093E20342
:1022200005910093E30305910093E4030491009367
:10223000E503FF91EF9120E10E94ED2D0E944B2ECE
:102240000091EB030395083009F400270093EB039A
:1022500000912C010C3019F41FEF1093A7020830E5
:1022600019F43FEF3093A402302F000F1127A2E999
:10227000B4E0A00FB11F0091780010917900119681
:102280003F93373084F411971D900C90332723E04F
:10229000200D311D0217130734F4900122503040F5
:1022A0000217130714F40C931E933F9133953F309C
:1022B00021F433270FEF0093AF0230932C0107E096
:1022C00030170CF4032F00937C0000913801087F35
:1022D000132F17501770012B00933801086010E47A
:1022E0000E94F5330FED00937A000091E004007135
:1022F00009F046C0009111040A3009F041C0009174
:10230000340106FF3DC001EC0E94453400913801C4
:1023100010E40E94F5330FEF08B9002707B90E94B7
:102320005D34009311010E945D34009312011091FD
:10233000110100911201000F111F000F111F000F5A
:10234000111F9801000F111F020F131F20E030E032
:1023500010F42FEF3FEFB9E40B0FB0EC1B1FB7E306
:102360002B1FBFE03B1F3093E2032093E303109346
:10237000E4030093E50320E10E94ED2D0E944B2E23
:10238000BF91AF913F912F911F910F911F900F908F
:10239000FFBE1895FFB620905A02222089F00F92B6
:1023A0001F920F931F932F93EF93FF9322240E946A
:1023B0008D31FF91EF912F911F910F911F900F90F1
:1023C000FFBE189500E10EBF0FEF0DBF00E002B990
:1023D000002701B90EE405B90093300103EF04B9F9
:1023E0000FEF08B9009507B90FE00BB90093310161
:1023F00002EF0AB9A0E0B1E0E2E7F8E0EA1BFB0B6C
:1024000000270D933197E9F70FEB009334010FEF9D
:102410000093320100933A01209138012F7B009301
:102420003801B5E7A0E3B0931404A093150400931A
:10243000EE030093250101E000938402009328023B
:102440000093CB030FE70093A3060AEA00939204DC
:102450000093930400E8009338010093F30308E02D
:10246000009339010AE000937F0200938202E0E7C3
:10247000F5E0A8E4B1E005E10E94A834E6E8F5E063
:10248000ADE5B1E007E20E94A834E2EDF5E0ACE989
:10249000B1E00DE00E94A834E0E2F6E0A4E8B1E08B
:1024A0000DE00E94A834EEE2F6E0A0EBB2E00DE011
:1024B0000E94A834EEECF4E0A4ECB2E00EE00E943E
:1024C000A834E0ECF4E0A6E2B3E00EE00E94A83409
:1024D000E6E5F6E0A4E3B3E007E10E94A834ECED02
:1024E000F4E0A3E5B3E00CE00E94A834EAE4F6E0EF
:1024F000A1E7B3E00BE00E94A834EEE6F6E0A4E921
:10250000B3E00FE00E94A834EEE7F6E0A3EAB3E000
:1025100007E10E94A834E2EDF6E0ACEBB3E00CE09A
:102520000E94A834EAE4F7E0AFEEB7E00CE00E94C6
:10253000A834E2E3F7E0ABE0B8E007E10E94A8349A
:1025400000913901016010E50E94F53300913901D5
:102550000E7F10E50E94F53304E11DE128E20E94A0
:10256000713404E11DE120E20E9471340AE41EE1AD
:1025700028E20E9471340AE41EE120E20E947134D4
:1025800000271FE128E20E94713400271FE120E2AA
:102590000E94713400E410E228E20E94713400E4E9
:1025A00010E220E20E94713401E020E10E942A340E
:1025B00001E028E30E942A3401E020E30E942A344B
:1025C00001E028E10E942A340E944B2E002707B91F
:1025D000009508B9F4E0E0EBD1E0C1EEBB27AA27F3
:1025E0000E943731019311962197D1F70E944E3501
:1025F00000270093DA043327222711270091D10402
:102600005FEF48E00E944F2E0091B80100937D03D8
:102610000093E9030091B90100937E030093EA035C
:1026200011270091CE0403FD10E81093330110E050
:102630000E94C6340E7000931004102F0091CE0437
:1026400003FD1091B1041E70109311041127009125
:10265000BD0407FD18E000FD1460109335010E94D1
:10266000D73403701127002339F012E0013021F034
:1026700011E0023009F013E01093330101E30093FD
:1026800012040AE00093F80308E0009397060CE4B4
:10269000009398060BE40093990600E400939A06D1
:1026A000002700939B0600939C060091D8040078B5
:1026B0000093F20391F404E1009347010FEF0093BC
:1026C00027020093E1030093C90300935103009391
:1026D0008B0200936402009308040091E50415E066
:1026E000019F800123E033270E946F4400930D0473
:1026F00010930C040091E0040C700093F403BB27CA
:10270000AA27002351F0BDEDA0ED043031F0BBEB62
:10271000A0EA003111F0B7E7A0E4B093F503A0936D
:10272000F60303E000937C000CED00937A00002791
:102730000093C5001091D70407E6112351F003E37D
:10274000113039F009E1123021F000E1133009F0C5
:1027500008E00093C40008EB0093C10006E000937A
:10276000C2000091E704002319F001E80093A502DC
:1027700000EE06BD05E005BD01E000936E000FE32D
:102780000093690007E00DBBB3E0A8EE1B9902C0FF
:102790001197E1F700913801086010E40E94F533C9
:1027A00000270E9445340E9445340E9445340E940F
:1027B00045340E9445340E9445340E9445340E94AD
:1027C00045340E9445340E9445340AEA0E9445344B
:1027D0000091380110E40E94F5330FEF08B900278B
:1027E00007B90E945D34053529F00CE100935D02C4
:1027F00000935E02789400915E02002309F0FACF04
:102800000091AF020023B1F300919F02002381F4F5
:102810000091DA040023A9F0F8940FEF00939F02CF
:10282000B3E1A8E8B0939D02A0939E02789409C0FA
:10283000F894B0919D02A0919E02109711F40C940F
:10284000007E0091F2030023E9F000910A08109144
:10285000EE03012BB9F4B7E0AFE4F7E0EBEF1CE0D7
:102860000D9101931A95E1F7B9E0A4ECF894B093B7
:102870000808A0930908789408E1009307080FEF6F
:1028800000930A08F894B0911404A0911504BA2B8F
:1028900059F4209138012F7B10E40091DF0400747B
:1028A0000127022B0093380178940E94EC350091A7
:1028B00092030023D9F44091930340FF17C00CE426
:1028C0001FE623E63BE647FF03C000E2102F980116
:1028D00000939F031093A0032093A1033093A203BE
:1028E0000FE00093920300270093930300910304E9
:1028F0000023FAF40091220017E1019F02E7000D86
:102900001091AF041017A8F0F89400270093F90372
:102910000093FA030395009303042091AE0204E5AB
:1029200016EA0E9488302091AD0204E515EA0E9463
:1029300088300091F30300FFAFC00E7F0093F303D4
:1029400007FF60C001E00093CB0303E00093CA03DC
:102950002091AE0204E516EA0E9488302091AD0273
:1029600004E515EA0E94883000919A020093E80479
:1029700004E11DE128E20E94713404E11DE120E23E
:102980000E94713401E020E10E942A3401E028E332
:102990000E942A3401E020E30E942A3401E028E169
:1029A0000E942A340E944B2E0091410110EC0E949B
:1029B000113400913B0110E70E9411340091420153
:1029C00010ED0E9411342091EB0410E50EE90E94F5
:1029D0008830BB27AA270091E0040C700093F40311
:1029E00051F0BDEDA0ED043031F0BBEBA0EA0031B9
:1029F00011F0B7E7A0E4F894B093F503A093F603C1
:102A000078944AC000270093CB0303E00093CA03E5
:102A1000222704E516EA0E948830222704E515EAF9
:102A20000E9488300091E80400939A0200270093E6
:102A3000E80407E128E20E94713407E11DE120E289
:102A40000E94713404E020E10E942A3404E028E36B
:102A50000E942A3404E020E30E942A3404E028E1A2
:102A60000E942A340E944B2E009141010C7F10ECF1
:102A70000E94113400913B012B7F10E70E9411341A
:102A80000091420100640F7D10ED0E9411342FEF80
:102A900010E50EE90E9488300091C9030023F9F087
:102AA0000091C8030023D9F400270093C9030091C3
:102AB0000304002311F003E50DC00091040400237A
:102AC00011F00DE407C00091B0040550F2F70A5F61
:102AD00010E3010F0093C7030CE00093C80330918B
:102AE00087020091A702002309F473C0F89400271D
:102AF0000093A7021091AA040091AB047894169554
:102B00000795169507950C3D08F063C0033C30E02F
:102B100098F431E0053A80F432E0073868F433E0A5
:102B2000093650F434E00B3438F435E00D3220F43B
:102B300036E00F3008F437E030938702363099F0F2
:102B400000910B04002309F044C0002700930904FE
:102B5000E2E3F7E0ABE0B8E007E10E94A83407E168
:102B600000930B0436C0343041F00091030400237D
:102B700021F00027009303040BC0353051F1009180
:102B80000404002331F10027009304040E94EE4462
:102B900010E00E94C6343091FD033E933E703093A6
:102BA00010040091CE0403FF309311042091FE0322
:102BB0001091FF030091000411962D931D930C9327
:102BC0000FEF0093C903009351030093E1030093B7
:102BD00027020091C302002309F4F9C000270093E3
:102BE000C3020091D001002309F0DCC030918702BC
:102BF00034300CF4C5C0343009F41DC0353009F44C
:102C0000A0C0363009F0E3C000910904002341F46C
:102C100000910A040E9419450FEF00930904D7C0E0
:102C20000091110404300CF0D2C000910A04039505
:102C30000093F103CCC0F894009103040095009335
:102C400003048AF001E0009303042091AE0204E53E
:102C500016EA0E9488302091AD0204E515EA0E9430
:102C600088307894B4C00E3F71F010E00E94C634F2
:102C70000093FD030D910093FE030D910093FF035C
:102C80000D910093000478940091D504002309F07D
:102C90000BC0F8940091D3040093D10478940E945F
:102CA0004E350E94194423C00091D50422271AE012
:102CB0000130C9F014E60230B1F023E018EE033021
:102CC00091F027E210E1043071F02AE318E90530B1
:102CD00051F02EE410E2063031F021E618EA073018
:102CE00011F023EC10E52093FB031093FC030091FB
:102CF000D604222712E3002361F01DE7013049F0DA
:102D00001AEF023031F021E014EF033011F029E026
:102D100014ECF8942093F9031093FA032093010420
:102D2000109302047894222704E516EA0E94883062
:102D3000222704E515EA0E9488300FEF0093C903AB
:102D400046C010E00E94C6340093FD030D9100932D
:102D5000FE030D910093FF030D9100930004009179
:102D60000404002319F00E94194431C00FEF0093AE
:102D700004040093C9030E944E350E94813527C088
:102D800000914C02009500934C020AE210E211F00F
:102D900000E21AE200933F03109348030FEF009301
:102DA000510315C00091CF010D3011F00E3079F4B0
:102DB0001091D10116305CF00091EF0303950C30B7
:102DC00009F400270093EF030FEF0093EC03009149
:102DD000340106FF06C00E9486460E94A4460E9457
:102DE0000847F8941091A4040091A5047894000F6A
:102DF000111F00930C0110930B010091CE0406707B
:102E0000043029F0063019F00027112714C0F89477
:102E10001091AC040091AD047894000F111F000FC5
:102E2000111F000F111F000F111F000F111F33275B
:102E30002AE00E946F440093080110930701F89460
:102E40001091A6040091A704789416950795009315
:102E50000A0110930901F8941091A8040091A904A3
:102E6000789416950795222733274091CE04542F46
:102E700040774032D9F456705630E1F013E30091B8
:102E80006902109F8001332720916402222309F4F4
:102E900023950E946F44073608F007E600936C0301
:102EA0003327222714E6019F800104C0202F312FF1
:102EB000002711270093100110930F0120930E019A
:102EC00030930D0122270091340106FD2068009106
:102ED000110404302CF00A3009F42062206404C08C
:102EE00000910F0400FD206200913A0105FF20616E
:102EF0000091CF04007306950695202B1091D00405
:102F00001370212B2093A602209139012971009181
:102F1000EA040078202B0091F303009500780695D1
:102F20000695202B00919902202B10912501112349
:102F300021F410913901211741F0F89420933901BF
:102F4000022F10E50E94F53378940091CE040670AC
:102F500009F4DAC100918D022091C8041091250175
:102F6000112311F4021731F020938D0212E008E5CD
:102F70000E94883022270091E00407FD2FEF009186
:102F80001104083009F42FEF00912501002321F4EA
:102F900000919302201731F02093930211E008E58D
:102FA0000E9488300091CE040078B9F0F894109116
:102FB0009604209197047894169527951695279551
:102FC00000912501002391F430917302231729F019
:102FD000209373020027009375020091750200FD93
:102FE0002091740200917202021731F02093720254
:102FF000112708E50E94883020917C020091CE04C0
:10300000007851F0F89430919E0420919F047894B8
:103010003695279536952795369527953695279594
:103020003AE7230F0091E00405FF05C02093EC046C
:103030000E94AD3420C000912501002391F400913D
:10304000CE04007849F030917B02231729F02093B9
:103050007B02002700937D0200917D0200FD2091FC
:103060007C0220937A0200917A02021721F016E581
:103070000EE90E948830009111040430A4F00A3057
:1030800091F0083081F02091E204009125010023A5
:1030900021F400918502201731F02093850214E578
:1030A0000EE90E948830209167020091CE040078DA
:1030B00051F0F89430919C0420919D0478943695B9
:1030C0002795369527950091E00405FF0BC02195C3
:1030D0002A3F10F4263308F4F7C02093EB040E9433
:1030E000AD34F2C026951091CE04107849F01091BD
:1030F0006602121729F020936602112710936802C6
:103100001091680210FD209167020091640202177D
:1031100029F400912501002309F430C020936402B2
:103120000091C102002351F546E00091CE040670E3
:1031300019F0023009F047E033272227009164029A
:103140001AE0019F800155270E944F2EADEBB2E09F
:103150000091B6010D930091B7010D930091B80154
:103160000D930091B9011091CE04167019F0123030
:1031700009F000E20C9301E10093C10200913401D7
:1031800006FD04C0002700936902BEC00091E00460
:1031900006FF9AC000911104003029F0023019F0A6
:1031A0000A3009F01CC0F89400913801086010E45E
:1031B0000E94F53305EC0E9445340091380110E47B
:1031C0000E94F5330FEF08B9002707B90E945D345C
:1031D0007894002321F400270093690295C0109190
:1031E000A302112319F0123009F08EC000270093BA
:1031F000A302109121010091220133272AE040917E
:10320000CE04467019F0423009F024E60E946F4463
:10321000009369021091640216C0309169033A511B
:1032200090F041E1349F80012AE033270E946F44EF
:10323000109164023FE7301B37FD3327009169028C
:10324000311708F4132F21E0101B19F40093A20288
:103250005BC010F4119521953091F803131718F401
:103260000093A20251C000270093A2021091EB0428
:10327000121B1A3F68F4163328F01093EB040E94D7
:10328000AD3422C019EF1093EB040E94AD3405C099
:1032900016E31093EB040E94AD341091EC04120F6E
:1032A0001A3B68F41A3728F01093EC040E94AD34EE
:1032B0000BC019EB1093EC040E94AD3405C01AE763
:1032C0001093EB040E94AD34442700919C0220919E
:1032D000EC04021739F020939C0212E50EE90E94DB
:1032E00088304FEF00919B022091EB04021739F0D8
:1032F00020939B0210E50EE90E9488304FEF442393
:1033000019F001E00093A3027894009110040A30B0
:1033100011F420EC3FC00091CE040078C1F0F89485
:103320001091980400919904789498013695279506
:103330003695279530917702321729F0209377023E
:103340003327309379023091790230FF07C011277B
:1033500000917802000F111F000F111F10950095AA
:1033600013702BEE35E0020F131F2091DB0433277F
:10337000220F331F220F331F220F331F220F331F41
:10338000200F311F36952795369527953695279529
:10339000369527950091CF04087031F4F894009188
:1033A000130400230AF420EC789400917602109123
:1033B0002501112311F4021731F02093760214E154
:1033C0000EE90E9488300091CE04007899F0F894BC
:1033D00030919A0420919B047894369527953695E0
:1033E000279530916F02231729F020936F02002751
:1033F000009371020091710200FD209170022695E8
:103400002695269500912501002321F400916E0256
:10341000021751F020936E0200E515EA0E948830F1
:1034200000E516EA0E9488300091CE04007899F0F9
:10343000F8943091940420919504789436952795CA
:103440003695279530916B02231729F020936B0254
:10345000002700936D0200916D0200FD20916C0227
:1034600026952695269500912501002321F40091AB
:103470006A02021751F020936A0202E515EA0E94DF
:10348000883002E516EA0E9488307894112700916E
:10349000370102FF13C003FF22C02091AE02222396
:1034A00021F42FE12093AE021FEF2091AD022223E1
:1034B00031F52FE12093AD021FEF21C02091AE0224
:1034C000222321F022272093AE021FEF2091AD028C
:1034D0002223A9F022272093AD021FEF10C02091D4
:1034E000AE02222321F42FE12093AE021FEF2091A0
:1034F000AD02222321F022272093AD021FEF00917D
:103500002501002311F4112361F02091AE0204E59E
:1035100016EA0E9488302091AD0204E515EA0E9467
:1035200088302091CE04207899F0F894309192045C
:103530002091930478943695279536952795309168
:103540006102231729F02093610200270093630290
:103550000091630200FD2091620200912501002389
:1035600049F4009160021091630210FD0091620223
:10357000021731F02093600216E10EE90E948830B4
:10358000789420918702222329F44091510240939C
:103590005203CFC024300CF47AC0243009F443C065
:1035A000253009F1263009F0C4C000910A041091B9
:1035B0005102112331F032F40A95002342F409E05C
:1035C00006C0B7C0102F03950A300CF000271091E9
:1035D0000B04112321F400930A040E9419450027CB
:1035E00000935102A6C0F8940091D10410915102A9
:1035F000112339F03AF40F770A9500234AF404E5D1
:1036000007C097C0102F0F77039505350CF00027E2
:103610000093D10478940E944E350E948135002792
:103620000093510286C0F8940091D6041091510283
:10363000112389F02091D001222309F023C0112306
:1036400022F40A954AF4002707C00395043024F0B9
:1036500019F004E001C06DC00093D604222712E3E4
:10366000002361F01DE7013049F01AEF023031F01C
:1036700021E014EF033011F029E014EC2093010451
:1036800010930204002700935102789452C00091D5
:10369000C202002309F04DC040914C020091540237
:1036A000442311F00091550240915102442329F026
:1036B00012F0039509C00A9507C02091560227FF12
:1036C00038C02F772093560212E3213021F014E600
:1036D000223009F01AEF002372F40C3E0AF40CEECB
:1036E0000195019F0094109411E0010E10E0111E4D
:1036F0001FEF019505C005310AF004E1019F112774
:1037000040914C02442359F4009354021093D9037E
:103710001093DA031092DB030092DC030AC00093DB
:1037200055021093DD031093DE031092DF03009225
:10373000E0030E94D734212F1C7116951695312F66
:1037400000911004083009F430622076203039F0FE
:10375000203419F0203639F007C0386005C0043035
:103760001CF0386001C030611091CF04187011F066
:10377000306407C010911304112311F03F7B01C086
:1037800030641091CE04117009F030680091250169
:10379000002321F410913D01311731F030933D01A8
:1037A000032F10E90E94113420EA009110040A301E
:1037B00019F42F7D206500C0009152030023B1F061
:1037C0001091500240914C0240FF10914F02010FA6
:1037D00012F403E003C004300CF00027442319F076
:1037E0000093500212C000934F020FC010E00E94DD
:1037F000C634007F0295102F037000934F02012FF3
:10380000069506950370009350021FE000914F0249
:10381000100F0E94B434083031F4002700934F0297
:103820001FE00E94B434332710914D02101719F095
:103830003FEF00934D021AE0019FECE7F0E0E00D4E
:10384000F11D3596A2E4B3E005910D9305910D931A
:1038500005910D9305910D931596BF93AF933F93EB
:1038600013E100915002100F0E94B4340D3031F476
:1038700000270093500213E10E94B4343F9110914D
:103880004E02011719F03FEF00934E02AF91BF9126
:103890001AE0019FECE1F2E0E00DF11D3596059193
:1038A0000D9305910D9305910D9305910D93009145
:1038B0005103032B51F000915003002331F40CE12C
:1038C0000093500300270093510300915002000F12
:1038D000000F10914F02102B1F93009152030023F1
:1038E00099F000270093520310E00E94C6340F7035
:1038F0001F911F931295012BF8940E930E94AD34E3
:1039000078940FEF0093E1031F91212B0091250183
:10391000002321F410913E01211731F020933E0144
:10392000022F10EA0E9411340091C202002309F014
:1039300071C00091370106FF6DC000915102002354
:1039400021F000270093510208C00091E1030023F9
:1039500009F460C000270093E10340914D020AE2A0
:10396000409FECECF0E0E00DF11DA2EDB2E00AE2C8
:103970000E94A83440914E020AE2409FEEE9F2E034
:10398000E00DF11DACEFB2E00AE20E94A834009114
:1039900054021091D802100F1093D8021091DC023B
:1039A000100F1093DC021091E602100F1093E60244
:1039B0001091EA02100F1093EA021091F402100F16
:1039C0001093F4021091F802100F1093F802009176
:1039D000550210910203100F109302031091060379
:1039E000100F1093060310911003100F1093100383
:1039F00010911403100F1093140310911E03100F55
:103A000010931E0310912203100F1093220300E75E
:103A10000093C202009191030023E1F41091CE04BF
:103A20001077129500912501002329F400918B0253
:103A3000011709F40FC010938B020AE0019FF4E014
:103A4000E8EEE00DF11DB3E0AFE50E94A83406E119
:103A5000009391030091CE040077003009F420C058
:103A6000003109F42BC0003209F436C0003309F4E8
:103A700036C0003409F436C0003509F436C00036CB
:103A800009F436C0F8941091A6040091A704789424
:103A90002CE333270E946F44202F00936F033FC015
:103AA000F8941091A4040091A50478942AE0332797
:103AB0000E946F44202F00936E0331C0F894109140
:103AC000A8040091A90478942AE033270E946F4447
:103AD000202F00936D0323C020916C0320C0209100
:103AE00069031DC020916A031AC020916B0317C09F
:103AF000F8941091070100910801789416950795A4
:103B00001695079516950795169507951695079599
:103B10002AE033270E946F4400937003202F009106
:103B20002501002321F400918A02021731F020932D
:103B30008A0210E10EE90E9488300091CE040670DE
:103B400009F404C1009111042227043064F0083004
:103B500074F0A9F00A3049F420610E94D734007251
:103B6000A9F0206813C0206811C028690FC0206127
:103B70000E94D734007209F02068286007C02062D4
:103B80000E94D734007209F0206828601091CE049A
:103B90001670163009F42460216000911104109110
:103BA0000F0417FF2E7F2F930E94E3343E91317054
:103BB00011962D911D910C9170E06EE154E840E852
:103BC0000E949B342F910CF422600091CE04007768
:103BD000003209F4206400912501002321F41091A2
:103BE0003B01121731F020933B01022F10E70E9496
:103BF00011340E94E3343E91317011962D911D9144
:103C00000C91882740913B0141FD1CC070E06BE5A1
:103C10005DE840E80E949B3414F4806113C070E0BA
:103C200067EB5BE140E00E949B3414F480620AC0C1
:103C300071E061E35DE240E80E949B3414F480642B
:103C400001C0806870E066E255E240EA0E949B3461
:103C500014F421E049C070E06CE45BE440E40E94AD
:103C60009B3414F422E040C070E063E55CEE40E673
:103C70000E949B3414F4222737C070E062E750E7BB
:103C800040EE0E949B3414F423E02EC070E067EBFA
:103C90005BE140E00E949B3414F424E025C070E016
:103CA00064EF54E240E00E949B3414F425E01CC011
:103CB00071E061E35DE240E00E949B3414F426E091
:103CC00013C071E06FE451EB40E80E949B3414F4A0
:103CD00027E00AC071E06BEA5FE340E00E949B349A
:103CE00014F428E001C029E0822B00912501002373
:103CF00021F410913C01811739F080933C01F89434
:103D0000082F10E80E9411348695869586958E714D
:103D100009F4816080640091CE04067021F00230C5
:103D200011F080628F7B0091F30300950078802B67
:103D300000912501002321F410914201811731F0F7
:103D400080934201082F10ED0E9411340E94E33449
:103D5000222713960C91087009F020683FE744274A
:103D60000091320105FF61C0822F0E911E912E91AC
:103D70003E913170110F221F331F442755276EE1EA
:103D8000B4E0AAE10EE1061B000F000F1127A00FFF
:103D9000B11F1D9117FD04C050FF962F5FEF11C09A
:103DA00013700D910217130761F40D911C91712F7F
:103DB000782777FD06C04FEF0093A4061F77109376
:103DC000A3066A95E9F650FF9EE10091340106FFD3
:103DD00027C00091D90402FF04C00B7F0093D904CF
:103DE00002C04423E9F42F933F938F939F930E9443
:103DF00064459F918F913F912F91B4E0AAE10EE12C
:103E0000091B000F000F1127A00FB11F30683D9351
:103E10002D930091A4060D930091A306082B0C93FB
:103E2000282F3091A3064091A40664E057EA46FD8E
:103E300002C05A50604045FD02C05451604044FDEC
:103E400002C05752604043FD02C05255604042FDDF
:103E500002C05659604041FD02C05A54614040FDC5
:103E600002C05053624060931B0150931C010091AB
:103E7000D9040D7F47FD02600093D90466E258EE35
:103E800036FF02C05651604035FF02C052536040B9
:103E900034FF02C05A58604033FF02C0565262409D
:103EA00032FF02C0585D644031FF02C05E566A4076
:103EB00030FF02C05A5A644160931D0150931E01A5
:103EC000232B00912501002321F410914401211797
:103ED00031F020934401022F10EF0E941134242F5F
:103EE00000912501002321F410914301211731F0A5
:103EF00020934301022F10EE0E94113480E10091C3
:103F00003701037049F0023029F0013039F4846040
:103F10008F7E04C0816001C0836080620E94D734BC
:103F20000C7F1127803139F01395843021F01395DF
:103F3000813309F01395012B0E93007109F0806411
:103F40001091CF04187009F0806410E00E94C6340C
:103F5000302F31702D911D910C9170E069E150EF7F
:103F600040EA0E949B340CF08068009125010023F8
:103F700021F410914101811741F0809341010E9489
:103F8000AD34082F10EC0E9411342091DD04009113
:103F90003D01007211F42091DC0400912501002301
:103FA00021F400918902021731F02093890212E175
:103FB0000EE90E9488300E94D734007419F080E81E
:103FC0009FE76AC088279FEF10E00E94C634302F19
:103FD00031702D911D910C9170E06BE157E740E439
:103FE0000E949B3414F49B7F57C070E06DE256EC46
:103FF00040EC0E949B341CF484609B7F4DC070E0B9
:104000006DE359E040E00E949B3414F4977F44C074
:1040100070E066E65FEF40E30E949B341CF488602A
:10402000977F3AC070E069E854E540E40E949B3411
:1040300014F49F7E31C070E060EA57E340EA0E94CA
:104040009B341CF480619F7E27C070E06FEA59E7C3
:1040500040EE0E949B3414F49F7D1EC070E064EF1C
:1040600054E240E00E949B341CF480629F7D14C0A7
:1040700071E061E35DE240E00E949B3414F49F7BB9
:104080000BC071E06DE758E740E40E949B341CF4DC
:1040900080649F7B01C09F7700912501002341F43C
:1040A00000913F01081721F400914001091761F0C8
:1040B00080933F0190934001082F10EB0E94113430
:1040C000092F10EB0E94113422270091C704109190
:1040D0008C02011719F02FEF00938C020091C90494
:1040E00010918E02011719F02FEF00938E020091AC
:1040F000CA0410918F02011719F02FEF00938F025D
:104100000091CB0410919002011719F02FEF00934A
:1041100090020091CC0410919102011719F02FEF39
:10412000009391020091CD0410919202011719F0B1
:104130002FEF009392020091D8040F711091880222
:10414000011719F02FEF0093880200917F02109160
:104150007E02011719F02FEF00937E020091820278
:1041600010918102011719F02FEF00938102009145
:10417000E80410919602011731F02FEF0093960298
:1041800003E00093CA030091F103002309F02FEF2D
:104190000091A60210919402011719F02FEF0093DD
:1041A00094020091E60410919502011719F02FEF87
:1041B0000093950200912501202B29F40091ED0335
:1041C000002309F478C0F8942F9300913801086017
:1041D00010E40E94F5330091ED03002369F00AED2D
:1041E0000E94453410EAD7E0CFE409910E9445349B
:1041F0001A95D9F71093ED032F91222309F451C09A
:1042000005ED0E9445340091C7040E944534009199
:10421000C9040E9445340091CA040E9445340091AB
:10422000CB040E9445340091CC040E944534009197
:10423000CD0403950E9445340091D8040F7111F00C
:1042400014E0010F0E94453400918002002311F018
:1042500000917F020E94453400918302002319F0EF
:104260000091820203950E944534009196020E94BB
:1042700045340091F103003839F402E00093F10372
:104280000A950E94453405C00E94453400270093DA
:10429000F1030091A6020E9445340091E6040E94B9
:1042A000453478940091080810910908012B19F4FD
:1042B000002700932501009111040A3021F4009198
:1042C000340106FD31C2F89400913801086010E411
:1042D0000E94F5330091EE030023D9F004EC0E9414
:1042E00045340091380110E40E94F5330FEF08B90E
:1042F000002707B910EAD7E0CFE40E945D340993A4
:104300001A95D9F71093EE030E945D340093E904E7
:104310006EC002EC0E9445340091380110E40E9406
:10432000F5330FEF08B9002707B90E945D340093F9
:104330001F010E945D34009320010E945D340093B0
:1043400015010E945D34009316012091CE042F7751
:104350001091150117FD20682093CE041F7710934C
:10436000150127FD14C00FEF00936302009368024C
:1043700000937D0200936D02009371020093750219
:1043800000937902009380020093830230C0309141
:10439000970220912001231791F020939702332751
:1043A00030938002222309F423E114E003E90E9400
:1043B0006F44F89400931A01002700931901789430
:1043C00020911F0100919802021789F03327309342
:1043D000830220939802222309F420E21AE702E1E3
:1043E0000E946F44F8941093170100931801789479
:1043F00010911501009116012091A5022F7B16FD49
:1044000020642093A5021F7326FF18C020FF16C04A
:104410002E7F2093A502F8941F930F9300913801EB
:10442000086010E40E94F5330FED0E9445340091BE
:10443000A5020E9445340F911F917894209132017A
:1044400026FD72C1169507951695079511E0013363
:1044500010F112E00134F8F013E00135E0F014E05F
:104460000136C8F015E00137B0F016E0013898F0D9
:1044700017E0013980F018E0013A68F019E0013BDB
:1044800050F01AE0013C38F01BE0013D20F01CE048
:10449000013E08F0112700919E06002309F044C157
:1044A00000919D06002351F4112309F43DC11BE046
:1044B00010939E06039500939D0636C1013039F492
:1044C0000091CC010130C9F0023059F0D2C0112363
:1044D00009F02AC11BE010939E06002700939D0659
:1044E00023C11B3009F417C11C3021F4112710938C
:1044F000CC0111C11093F1030EC1113031F400272A
:104500000093CC010E94EE4406C1123041F4F894AD
:104510001091340104E0102710933501FCC01330D2
:1045200041F4F8941091340108E0102710933501FC
:10453000F2C0143041F4F8941091320100E81027D1
:1045400010933301E8C0153019F40E941944E3C0F8
:104550001730D1F4F89410E00E94C634302F009345
:1045600091062D91209392061D91109393060D9123
:10457000009394064D91409395064C914F7E409345
:1045800096060E948135C7C0183051F5F89410E0A6
:104590000E94C634009197060E930E70009310048B
:1045A0001091CE0413FF0093110411960091980608
:1045B0000D93009199060D9300919A060D93009129
:1045C0009B060D9300919C060C930FEF009327021E
:1045D0000093E103002700935402009355029BC00F
:1045E0001930B1F4F89410E00E94C6340093970695
:1045F0000D91009398060D91009399060D910093EB
:104600009A060D9100939B060D9100939C0683C022
:104610001B3089F4F8940091D104102F0F77039583
:1046200005350CF00027F8940093D1040E944E3514
:104630000E94813570C01A3041F4F8941091320113
:1046400008E010271093330166C01C3009F063C0E6
:10465000F8940091D104102F0F770A9500230AF4E3
:1046600004E5F8940093D1040E944E350E948135F0
:1046700052C0113011F4002735C0123011F405E09A
:1046800031C0133011F40FE02DC0143011F404E1E7
:1046900029C0153011F409E125C0163011F40EE1DE
:1046A00021C0173011F403E21DC0183011F408E2E4
:1046B00019C0193011F40DE215C01A3011F40AE0D6
:1046C00011C01B3021F402E00093CC0124C01C3047
:1046D00011F501E00093CC01F8940E944E350E9440
:1046E000813519C0402F4B5F0093B0040E94D7342E
:1046F00017FD05C00091B00403950417A9F70FEF4B
:104700000093C9030093E10300932702002700935D
:1047100054020093550200919D06039500939D0657
:10472000F8940E94AD3478940091D103002369F588
:1047300011271093D1030091CF0300FF26C01093DF
:10474000CF031091D6032091D703021739F0112718
:104750001093D8030093D703102F09C02091D803DA
:10476000222329F4002312F0139513951A95109320
:10477000D60320912802121719F02195121729F457
:1047800011271093D6030093D1030091D203002385
:1047900069F511271093D2030091D00300FF26C0C2
:1047A0001093D0031091D3032091D403021739F052
:1047B00011271093D5030093D403102F09C0209123
:1047C000D503222329F4002312F0139513951A958B
:1047D0001093D30320912802121719F02195121774
:1047E00029F411271093D3030093D2030091D00131
:1047F000002309F09DC106E010912702112329F43E
:104800000091370106FD1FC00BE00093D501002782
:104810000093D1010093D6010FEF0093D0010091D6
:10482000CC01002371F0023061F000E200937C03C0
:1048300000937D0300937E0300937F0300E20093C7
:10484000AB020C94FA1300919901002309F078C08F
:1048500000913A0104FD2DC00FEF00939901F894E7
:1048600000913401037F00933401009335010095DA
:1048700000933A0110E60E94F533009132010F7760
:10488000009332010093330100950093370110E348
:104890000E94F5330FEF0093CC030093CD03002764
:1048A0000093CB010091CE04077F0093CE040C94BB
:1048B000FA1300919A01002309F008C000913A010F
:1048C00000FD24C30FEF00939A019EC40AE00093F9
:1048D00028024091D20340FF24C010E00E94C63459
:1048E000102F0E70069547FF04C00A9532F407E0BA
:1048F00004C0039508300CF00027000F009310044B
:104900002091CE0423FF00931104117F012B0E93FD
:10491000F89400270093D2030FEF009327027894B6
:1049200073C400913A0100FF6FC4002700939A01FD
:104930000093D3030093D50301E000932802E6C25D
:104940000AE0009328020091CC03002341F000917B
:10495000C801002321F40093CC030E94ED340091A0
:10496000CD03002341F00091C601002321F4009300
:10497000CD030E9408351091D10310FD1BC0F8949F
:1049800000913A0102FD0AC00091A902002311F032
:104990000C94FA130FEF0093A90221C003FD4BC042
:1049A0000091AA02002311F00C94FA130FEF009368
:1049B000AA0206C0F89429E01091D10317FF0FC096
:1049C0000091B0040A9500230AF401E30093B004B7
:1049D0000E94D73417FD12C02A9591F72CC0009180
:1049E000B0040395023309F400270093B0040E9439
:1049F000D73417FD03C02A9591F71DC010E00E941F
:104A0000C6340E70009310041091CE0413FF00936F
:104A100011040E94AD340FEF009327020093C903E5
:104A20000093E10300270093540200935502009382
:104A3000D1030C94FA134091D20340FF5FC047FFAB
:104A40001DC00091B0040023A1F0053091F00A30A0
:104A500081F00F3071F0043161F0093151F00E3105
:104A600041F0033231F0083221F00D3211F00A9595
:104A70001CC000270093D2030C94FA130091B004D9
:104A80000430B9F30930A9F30E3099F3033189F3F7
:104A9000083179F30D3169F3023259F3073249F3E2
:104AA0000C3239F3013329F303950F930E94D73465
:104AB0001F771C930F910093B0040E94D7341068A5
:104AC0001C9310E00E94C6340E70009310041091E5
:104AD000CE0413FF009311040E94AD340FEF009336
:104AE000C9030093E10300932702002700935402B7
:104AF000009355020093D2030C94FA1311270091EE
:104B00003A0104FF0EC01093990100270093D603C9
:104B10000093D3030093D8030093D50301E00093DF
:104B2000280200912702002309F44BC40C94FA13C5
:104B30000091D301002311F00C94FA131091D501C8
:104B4000112339F11A951093D5010091D6012091C6
:104B5000D101201710E029F420912702222309F423
:104B60001FEF2091CF010E943E2F0091D6010395A7
:104B700016E020912702222309F41BE0011709F413
:104B800000270093D6019093D4019093D3010C9405
:104B9000FA1300912702002349F00027009327020F
:104BA0000093D2010093D0010C94FA1300913701C5
:104BB00006FDEFC0112700913A0100FF1FEF10938F
:104BC0009A01112331F10091D20300FF0C940926C0
:104BD0001127109359021093EF031093F0031093D1
:104BE000D6011091CF01139507FD125022F011311B
:104BF0001CF0112701C010E11093CF010027009392
:104C0000D20306E00093D1010BE00093D5010C9490
:104C1000FA130AE010915902112321F00BE00093DE
:104C2000D5010AE0009328022091D10320FF2AC079
:104C300000270093D10300919A01002331F000274F
:104C400000939A010FEF00939B010091D10127FD82
:104C50000A9507FD0AE00093D6010091D101200FCB
:104C60000AE022F02B3000E009F0022F0093D1017E
:104C700002E00093D50100270093EF030093F003B7
:104C80000C94FA130091D20300FF0C94FA13F7E18D
:104C9000ECE91091CF0125E0129F22271091D1015C
:104CA0001630DCF1100D4091CF014D3069F04E30DF
:104CB00059F0193291F540910704442309F05DC081
:104CC0004FEF4093050429C04091F003040F43E5E2
:104CD00022F04427043509F0402F4093F0031FEFE2
:104CE0001093EC031091D10116500091CF010D509B
:104CF00025E0029F100D1F7012952227B7E0AFE448
:104D0000A10FB21F0091EF03A00FB21FF6E0EEED6E
:104D1000E40FF21F04910C9330C0110F221F110FEA
:104D2000221FE10FF21F15914591742F5591649147
:104D30000E94B434802F4A9512F00695FCCF209142
:104D4000D203052321F0061741F0020F09C02223E8
:104D50003AF0662329F0020F03C022230AF4020F5F
:104D60007A951AF0000F550FFBCF50958523082B2D
:104D7000F8940C930E94AD34789411271093D203C9
:104D800001E00093D5010091D1010093D6010C946C
:104D90000F2A00270093590210919A01112329F03C
:104DA00000939A010FEF00939B010091D101002322
:104DB00062F001E00093D5010091D1010093D6018A
:104DC0000FEF0093D1010C94FA130091D20100234C
:104DD000A9F40FEF0093D2010091EC030093ED03CF
:104DE000F5E0E4ECB1E0A7ED0EE00E94A8340EE09F
:104DF0000093D4010093D3010C94FA130091E504BD
:104E000015E0019F800123E033270E946F44009347
:104E10000D0410930C0400270093D2010093D001DD
:104E20000093EF030093F0030093D6030093D303A2
:104E30000093D8030093D5030093EC0301E00093A3
:104E400028020091D90400FF0FC00E7F0093D904FF
:104E500000270093A40618E7B4E0AAE10D931A9581
:104E6000E9F70FE70093A30610E00E94C6340E7026
:104E700000931004102F0091CE0403FD1091B10493
:104E80001E70109311040FEF009327020093E103AB
:104E9000009351030093640200938B020091CC01B4
:104EA000002399F0023089F00DE400937C03009117
:104EB000E90300937D030091EA0300937E030AE374
:104EC00000937F0300E20093AB020091E0040C70BA
:104ED0001091F403011711F40C94FA130093F403E6
:104EE000BB27AA27002351F0BDEDA0ED043031F01F
:104EF000BBEBA0EA003111F0B7E7A0E4F894B0935F
:104F0000F503A093F60378940C94FA130091C8016A
:104F1000002309F08EC00091CB0100FF23C00023C5
:104F20007AF400270093CB01F8940091CE04077F18
:104F30000093CE0478940E94ED340E94083579C025
:104F400000270093CB01F8940091CE0408600093F1
:104F5000CE0478940091B1040E70009311040E9465
:104F6000233567C0F8940091C70110913A017894F5
:104F700000FF03C00023C2F452C00091AA02002324
:104F800009F057C013FD55C00091CE04087009F414
:104F900050C01FEF1093AA020E94ED430E942335D8
:104FA0000FEF0093270245C00091BD0400680093F5
:104FB000BD0402E50093A7010AE30093A801209134
:104FC0004E012093A90110914F011093AA01009165
:104FD00050010093AB01009151010093AC0100918D
:104FE00052010093AD01009159010093AE0100916F
:104FF0005A010093AF0100915B010093B001009151
:10500000E104002341F00E94FB442093A801109387
:10501000A9010093AA0105E10093C80107C00E94FD
:10502000ED340091BD040F770093BD040027009379
:10503000C7011091CE040091C601002339F0187009
:1050400009F439C000270093CA01C4C0187009F4DC
:1050500021C00091A902002309F0BCC000270093E1
:10506000CA0100913A0102FDB5C01FEF1093A902D9
:1050700010E00E94C634F8940093B1040D9100939F
:10508000B2040D910093B3040D910093B4040E94F7
:105090002335A0C01091BD040091C901002359F02F
:1050A00012F0116003C00E9408351E7F1093BD04EA
:1050B00000270093C90100270093CA0140913A01DB
:1050C00043FD41C04FEF4093CA014091370147FD76
:1050D00020C00091A802002309F01BC00FEF00932D
:1050E000A802F8940091B5041091B604012B109118
:1050F000B704012B1091B804012B59F0002700933D
:10510000B5040093B6040093B7040093B8040E945A
:10511000AD340091D20300FF16C0F8943091B5046D
:105120002091B6041091B7040091B8040E94F32EA8
:105130003093B5042093B6041093B7040093B804D9
:105140000E94AD34789440913A0142FD5DC04FEF2A
:105150004093CA014091370147FD21C00091A80248
:10516000002309F01CC00FEF0093A802F8940091EF
:10517000B9041091BA04012B1091BB04012B1091BA
:10518000BC04012B61F000270093B9040093BA041A
:105190000093BB040093BC040E94AD34789400914A
:1051A000D20300FF31C0F8943091B9042091BA04C1
:1051B0001091BB040091BC040E94F32E0093BC0428
:1051C0001093BB042093BA043093B9040E94AD3409
:1051D00078941AC00091D20300FF16C0F89411E031
:1051E0000E94C6340170302F2D911D910C910E94A8
:1051F000F32E0C931E932E930E910E7F3170302B55
:105200003C930E94AD34789410E00E94C634302F55
:1052100031702D911D910D914091CE04487009F08F
:1052200039C04091AC02442309F034C04091CA0116
:10523000442309F02FC04091D20340FF2BC0F894C3
:105240000E94122F789488277727662754E640918A
:10525000DE04442309F05AE040913A0141FD08C0C0
:1052600067E250E14091DE04442311F063E058EE20
:105270004091D203442352F441E0509560957FEF72
:105280008FEF540F40E0641F741F841F050F161F1B
:10529000271F381F44274093D2034091AC02442378
:1052A00009F08FC09091D10390FD25C04091E80393
:1052B00040FD0BC047FD19C04091360142FD0CC0B6
:1052C000F89444604093360178949091E8039E7F6F
:1052D0009093E80391E00FC043FF02C00C94AB2908
:1052E000F89448604093360178944091E8034F77F2
:1052F0004093E8039FEF44274093D103F8940E9422
:10530000122F8827772766275AE04091DE0444232E
:1053100009F051E040913601427029F040913A0184
:10532000789441FD08C063E058EE4091DE044423C8
:1053300011F0662754E6992352F441E050956095A8
:105340007FEF8FEF540F40E0641F741F841F050F21
:10535000161F271F381F70E060E057E24FE0401B28
:10536000510B620B730B6AF571E069EC53EC40E88A
:10537000401B510B620B730B22F13F932F931F9332
:105380000F9310E00E94C634302F31702D911D9183
:105390000D914F915F916F917F91041739F415171B
:1053A00029F4261719F4371709F40BC0F8944E9313
:1053B0005E936E930E910E7F702B7C930E94AD34A2
:1053C000789410E00E94C634302F31702D911D91D9
:1053D0000D914091CE04487051F540913A0143FD42
:1053E00026C07091B5046091B6045091B704409105
:1053F000B804040F151F261F371F70E060E057E246
:105400004FE0401B510B620B730B4AF471E069ECE7
:1054100053EC40E8401B510B620B730B42F410E05D
:105420000E94C634302F31702D911D910D91882727
:1054300071E06BEA5EE34FEF401B510B620B730BA5
:105440000AF08FEF809307040F931F932F933F93DE
:10545000552745E00E944F2E0091F203002329F0CA
:1054600000910A08002309F47AC00091C5010023C5
:1054700009F075C0E2EBF1E0AEE4B1E089E0772736
:105480000091BB03002341F00091340106FD67C089
:1054900000270093BB0375E10C911191011759F09E
:1054A000813039F4003229F40091DE04002309F43C
:1054B00002C01C9375E111968A9521F0843061F742
:1054C0001696EACF0091DE04002319F410E210933F
:1054D0005C01209105041127772319F4222309F494
:1054E0003EC01093050475E10091E104002309F426
:1054F00034C07BE1222311F077E21FEF1093060402
:1055000020914E0110914F017F930E94FB447F91A7
:1055100020936F011093700100937101009150016D
:1055200000937D010091510100937E010091520191
:1055300000937F0100915A010093810100915B016A
:105540000093820100915C01009383010091DE04CD
:10555000002319F400E2009383017093C5013F9189
:105560002F911F910F9174E063E35EE048ED80910D
:10557000BE04882321F474E06CE25DE140E8809190
:105580001004883011F18A3001F174E063E356E1D0
:1055900048EA8091BE04882321F474E06CE25AE367
:1055A0004CEC80911004803081F0843071F08C30AC
:1055B00061F074E063E357E048E08091BE04882323
:1055C00021F474E06CE250E044E37F936F935F93C7
:1055D0004F93040F151F261F371F009322081093A7
:1055E0002308209324083093250840914D025AE067
:1055F000459FECE7F0E0E00DF11D772765915591AF
:1056000045913327222711270027809110048830E5
:10561000A1F08A3091F015910491843071F08C30B2
:1056200061F0803051F0009510952095309581E023
:10563000080F80E0181F281F381F400F511F621FDE
:10564000731F0F911F912F913F914F935F936F9312
:105650007F93041B150B260B370B7091D9036091B8
:10566000DA035091DB034091DC03041B150B260B7E
:10567000370B0093260810932708209328083093AF
:10568000290840914E025AE0459FECE1F2E0E00D1E
:10569000F11D33272591159105917727662755919F
:1056A000449180911004843069F08C3059F080303E
:1056B00049F0863089F08E3079F0823069F05527D4
:1056C00044270AC081E07095609550954095480F39
:1056D00080E0581F681F781F040F151F261F371FF3
:1056E0007F916F915F914F91040F151F261F371FF8
:1056F0007091D9036091DA035091DB034091DC0390
:10570000040F151F261F371F7091DD036091DE0304
:105710005091DF034091E003041B150B260B370B60
:1057200000932A0810932B0820932C0830932D08FF
:1057300040914E025AE0459FECE1F2E0E00DF11D90
:105740003327259115910591772766275591449127
:1057500080911004883049F08A3039F0803091F01F
:10576000843081F08C3071F017C000271127222778
:105770003327009332081093330820933408309372
:10578000350838C081E07095609550954095480F78
:1057900080E0581F681F781F040F151F261F371F32
:1057A0007091DD036091DE035091DF034091E003CF
:1057B000041B150B260B370B00933208109333088C
:1057C00020933408309335087727662750911701C6
:1057D0004091180180911004823041F0803051F4E2
:1057E00081E07095609550954095480F040F151F06
:1057F000261F371F00932E0810932F082093300880
:1058000030933108809111044DE730E023EA1FED19
:1058100003EB883029F14091E30430E023EA13EDF3
:105820000BEF8630E9F08E30D9F04DE730E023EA17
:105830001DE300E18A30A1F0803091F0823081F0E8
:105840004091E40430E023EA1DED0BE55091E004C3
:1058500057FF06C04091E40430E023EA0BE61BEE5C
:105860005527440F551F440F551F440F551F440F14
:10587000551F6627040F151F261F361F0093360875
:105880001093370820933808309339080E94E33486
:105890003E91317011962D911D910D9140913401E1
:1058A00044FD14C04091CE04487081F440913A0107
:1058B00042FD0CC07091B9046091BA045091BB04D0
:1058C0004091BC04040F151F261F371F0F931F9311
:1058D0002F933F938091340186FD04C08091E004B2
:1058E000807161F4709139086091380850913708DF
:1058F00040913608040F151F261F371F00933A08E2
:1059000010933B0820933C0830933D08882771E0B2
:105910006FE451EB40E80E949B340AF08260809370
:1059200099028091E004807109F056C03F912F9157
:105930001F910F910F931F932F933F93882771E02F
:105940006BEA5EE34FEF401B510B620B730B0AF0E7
:105950008FEF90910704892B809307040E9487445E
:10596000A6F0009111040430BCF10A30A9F10091B5
:10597000340106FD31C0002700933A0800933B082C
:1059800000933C0800933D0827C01091E00415FDEA
:1059900011C0002700933A0800933B0800933C088D
:1059A00000933D08009336080093370800933808A9
:1059B000009339080091BB03002371F40091340176
:1059C00006FF0AC00091BA03002331F407E10093F7
:1059D000BA030FEF0093BB03442736E0A2E2B8E01E
:1059E000CEE3D8E024E00D911991011709F0416050
:1059F0002A95C9F7440F3A95A9F7442309F48CC0B6
:105A0000F8944F9346FF13C00091220800933E087C
:105A10001091230810933F082091240820934008F8
:105A2000309125083093410848E20E94092E4F9199
:105A30004F9345FF13C00091260800934208109130
:105A40002708109343082091280820934408309198
:105A500029083093450840E20E94092E4F914F9348
:105A600044FF13C000912A080093460810912B08A8
:105A70001093470820912C082093480830912D0856
:105A80003093490848E10E94D22D4F914F9343FF34
:105A900013C000912E0800934A0810912F0810930C
:105AA0004B082091300820934C08309131083093F6
:105AB0004D0840E30E94D22D4F914F9342FF13C0F7
:105AC0000091360800934E081091370810934F0844
:105AD00020913808209350083091390830935108AC
:105AE00040E10E94D22D4F9141FF13C000913A082E
:105AF0000093520810913B081093530820913C08E2
:105B00002093540830913D083093550848E30E9493
:105B1000D22D0E944B2E78943F912F911F910F917F
:105B2000409199014423E1F540919A014423C1F544
:105B30004091CE04487021F440913A0142FD30C0BA
:105B4000552745E00E944F2E0091C601002341F5E4
:105B5000E2EBF1E0A1E9B1E088E077270C91119147
:105B6000011711F01C9375E111968A9509F0F6CF93
:105B70007093C60108E500938F010AE3009390013A
:105B80000091E104002361F02091910110919201B4
:105B90000E94FB4420939001109391010093920185
:105BA0000C94FA134F93332352F4009510952095DB
:105BB000309541E0040F40E0141F241F341F67E1BB
:105BC0005BED41E970910D04470F70910C04571F74
:105BD00070E0671F0E9446312F912F9301E00E94D1
:105BE0002A340091E2032F912F930E942A340091CE
:105BF000E3032F912F930E942A340091E4032F9105
:105C00002F930E942A340091E5032F910E942A3499
:105C100008954F93332352F40095109520953095B5
:105C200041E0040F40E0141F241F341F6EE050E5D4
:105C30004AE87091E504470F70E0571F671F0E9404
:105C400046312F912F930091E20314E00E947134AA
:105C50000091E3032F912F9315E00E94713400917E
:105C6000E4032F912F9316E00E9471340091E50315
:105C70002F912F9317E00E9471340091E6032F912A
:105C80002F9318E00E9471340091E7032F9119E0DF
:105C90000E94713408952F9A00002F9808955F9301
:105CA0004F9340E233235AF4309520951095009598
:105CB00041E0040F40E0141F241F341F4DE24F93B6
:105CC00044275527662778E183E090E3000F111FF2
:105CD000221F331F441F551F661F7A9589F1609359
:105CE0002F01680F63FF60912F0160932F01690FEF
:105CF00067FF60912F0150932F01580F53FF509170
:105D00002F0150932F01590F57FF50912F014093AE
:105D10002F01480F43FF40912F0140932F01490F5E
:105D200047FF40912F0130932F01380F33FF3091FF
:105D30002F0130932F01390F37FF30912F01C6CF3C
:105D40001F910F912EE2A1EBB1E01D93762F72957A
:105D50007F7070637D93013009F42D936F706063E1
:105D60006D93023009F42D93752F72957F707063D7
:105D70007D93033009F42D935F7050635D9304307D
:105D800009F42D93742F72957F7070637D930530A5
:105D900009F42D934F7040634D93063009F42D9311
:105DA000732F72957F7070637D93073009F42D9384
:105DB0003F7030633D93083009F42D935F91552374
:105DC00009F00895199721E03D91303349F4021705
:105DD00039F0129730E23D931D9323952930A1F7B6
:105DE00012971C9308954091AC02442309F0089542
:105DF0000E94122F7727662755274AE080913A01A3
:105E000081FD02C053E048EE8091D20388232AF43A
:105E1000041B150B260B370B0895040F151F261FA7
:105E2000371F08950F9300913A0101FD25C000919D
:105E3000E004037059F00130B1F0023069F005E779
:105E40000093A10600E30093A20613C0002700936D
:105E5000A1060093A2060DC00AE30093A10608E97B
:105E60000093A20606C003E10093A10608E8009390
:105E7000A20600270093AC020F910895422FE6E29C
:105E8000F6E1442309F440C0ECE3F6E14130E1F1EE
:105E9000E2E5F6E14230C1F1E8E6F6E14330A1F196
:105EA000EEE7F6E1443081F1E4E9F6E1453061F1F5
:105EB000EAEAF6E1463041F1E0ECF6E1473021F163
:105EC000E6EDF6E1483001F1ECEEF6E14930E1F0C3
:105ED000E2E0F7E14A30C1F0E8E1F7E14B30A1F050
:105EE000EEE2F7E14C3081F0E4E4F7E14D3061F0AF
:105EF000EAE5F7E14E3041F0E0E7F7E14F3021F01D
:105F0000E6E8F7E1403101F0043039F42091CF04A4
:105F1000287019F0F6E1EAE10DC0000F2227E00F2A
:105F2000F21F069535912491330F221FF8E0E6EF1A
:105F3000E30FF21FD1E0C7ED26E0922F35913993A0
:105F40002A95E1F72FE1299328E2299327E629935F
:105F500021E0299329939B5F112339F02FE12993A5
:105F600022E7299321E029939D5F2591222349F47B
:105F70003591309326012591299393953A95D9F738
:105F80002591043029F43091CF04387009F0B6C05F
:105F9000B7E1ACE935E0439F06300CF0000D442733
:105FA000000F441F000F441FA00FB41F359133236F
:105FB000EAF1FF93EF93FD014491EF91FF9140349B
:105FC000ACF04A349CF440544F704295B7E0AFE4D3
:105FD000A40F40E0B41F3CE02D91222329F0299327
:105FE00093953A95C9F78AC020E284C0442740932C
:105FF000CE031F93FF93EF93FD01159145915591AA
:1060000064910E94B4344A9512F00695FCCF0523A2
:10601000039FEF91FF911F91E00DF11D2591222328
:1060200021F0299393953A95C9F768C04FEF55270A
:10603000222312F444275FEF409359025093CE037A
:106040003195432F1F939F93CF93DF93FD01BB2780
:10605000A491552339F01A2F0E94B43433272227F4
:10606000112705C0B1E0332722271D910C91552738
:106070000E944F2EDF91CF919F911F910091260199
:1060800031E1301B313079F1323041F1333009F1F7
:106090003430D1F0353099F0363061F0373029F0B6
:1060A0000091B201099393953A950091B301099338
:1060B00093953A950091B401099393953A9500917F
:1060C000B501099393953A950091B601099393957B
:1060D0003A950091B701099393953A950091B801CB
:1060E000099393953A950091B901099393953A953F
:1060F00029F020E2299393953A95E1F7112339F09D
:106100000FE1099302E7099300E009939D5F089569
:10611000F8943091310130653BB93FEF37B9309198
:10612000390138B9439A449829980E9434310E9421
:106130003431299A0E943431449A29980E9434318A
:106140000E943431299A0E9434310E94343143989C
:1061500029980E9434310E943431299A0E943431A6
:106160000E9434310E3961F40E94E730012F0E9401
:10617000E730022F0E94E73000270E94E73008C076
:106180000E94E730012F0E94E730022F0E94E73083
:106190000E9434310E943431449A29980E9434314B
:1061A0000E943431299A0E943431439A29980E94DE
:1061B00034310E943431299A0E943431449829980C
:1061C0000E9434310E943431299A7894089538E03D
:1061D000449A000F08F4449829980E9434310E9490
:1061E0003431299A439A29980E9434310E943431DB
:1061F000299A0E943431439829980E9434310E9490
:106200003431299A0E9434310E9434313A9501F791
:10621000449829980E9434310E943431299A439A33
:1062200029980E9434310E943431299AC091310159
:10623000C062CBB9CC27C7B929980E9434310E94DB
:106240003431C6B1299AC0913101C065CBB9CFEFC5
:10625000C7B9C0913901C8B9439829980E9434310F
:106260000E943431299A0895000000000895F99998
:10627000FECFB2BDA1BDF89A00B50895F999FECF41
:10628000B2BDA1BD00BDFA9AF99A0895772770931F
:10629000E2037093E3037093E4037093E503709358
:1062A000E6037093E70340FD0E945D3166955795C4
:1062B000479573957631B9F7089588279927A32FC5
:1062C000B22FC12FD02FE72FEE2341F0DD0FCC1FCF
:1062D000BB1FAA1F991F881FEA95F6CFE091E7031D
:1062E000DE0FD093E703E091E603CE1FC093E603F1
:1062F000E091E503BE1FB093E503E091E403AE1F18
:10630000A093E403E091E3039E1F9093E303E091E5
:10631000E2038E1F8093E20308950091CE0400787B
:1063200041F5002700930708009347010093C5013A
:106330000093C8010093C6010093D3010093C102EA
:106340000093C202009391030093AB020093920367
:106350000093BA030093C8030093CA030093500349
:1063600000930B040093180400935C0200935D02F9
:10637000089501E010904501011509F488C10395C5
:10638000011509F4FFC10395011509F4C3C0039574
:10639000011509F4DCC00395011509F4E6C0039565
:1063A000011509F4F0C00395011509F4FCC003952B
:1063B000011509F406C10395011509F410C10395EF
:1063C000011509F41AC10395011509F424C10395B7
:1063D000011509F42EC10395011509F438C103957F
:1063E000011509F442C10395011509F4AFC10395E4
:1063F000011509F45AC10395011509F491C10395DA
:10640000011509F460C10395011509F47AC101E091
:1064100020900708222009F03AC10091F2030023DE
:1064200061F000910A08002309F4BBC1009108083B
:1064300010910908012B09F0B4C102E02090470136
:10644000222009F09FC103952090C501222009F068
:1064500061C003952090C801222009F078C00395FF
:106460002090C601222009F080C003952090D3011E
:10647000222009F088C003952090C102222009F053
:1064800092C003952090C202222009F09AC0039581
:1064900020909103222009F0A2C003952090AB0226
:1064A000222009F0AAC0039520909203222009F02F
:1064B000B2C003952090BA03222009F0BAC0039518
:1064C0002090C803222009F0C2C0039520905003F9
:1064D000222009F0CAC003952090CA03222009F0A7
:1064E00035C1039520900B04222009F0DEC00395EE
:1064F00020901804222009F013C1039520905C021B
:10650000222009F0E0C0039520905D02222009F0CE
:10651000F8C047C10093450104E1E8E4F1E01091BF
:10652000E104112359F0E9E6F1E00AE110910604D3
:10653000112321F01CE0010FE11BF0402090C50168
:106540002A942092C5010219102E44242EC10093D2
:1065500045012090C8012A942092C80104E1021943
:10656000102EECE9F1E0442420C100934501209075
:10657000C6012A942092C60104E10219102EE4E813
:10658000F1E0442412C1009345012090D3012A94E4
:106590002092D3010091D4010A950219102EE7ED43
:1065A000F1E0442402C1009345012090C1022A94E5
:1065B0002092C10200E10219102EE0EBF2E0442427
:1065C000F4C0009345012090C2022A942092C20296
:1065D0000FE60219102EE4ECF2E04424E6C000932A
:1065E0004501209091032A942092910305E102191C
:1065F000102EE3E5F3E04424D8C000934501209039
:10660000AB022A942092AB020FE10219102EE1E7AF
:10661000F3E04424CAC000934501209092032A94D9
:10662000209292030EE00219102EE4E9F3E04424D4
:10663000BCC0009345012090BA032A942092BA036B
:1066400006E10219102EE3EAF3E04424AEC0009301
:1066500045012090C8032A942092C8030BE0021938
:10666000102EECEBF3E04424A0C01091370116FF8C
:1066700098C000934501209050032A942092500323
:106680000BE10219102EE4E3F3E044248EC00093E2
:106690004501209007082A942092070807E1021973
:1066A000102EEFEEF7E0442480C0009345012090C7
:1066B0000B042A9420920B0406E10219102EEBE041
:1066C000F8E0442472C000934501112720905C0239
:1066D00027FE02C021941FEF2A9420925C0209E158
:1066E0000219102E043144F0112331F01394139445
:1066F0001394139413941394E6E9F6E0442440941D
:1067000054C00093450120905D022A9420925D02BE
:106710000BE10219102EE6EBF6E04424409445C04C
:1067200000934501209018042A94209218040BE04D
:106730000219102E0B3029F40091170405FD01C039
:106740001394ECE3F6E0442440942FC000934501F9
:106750002090CA032A942092CA0302E00219102E44
:106760000091E804000F000FE0E5F5E0E00F00E025
:10677000F01F0091CB03002311F4ECE4F5E0442476
:10678000409413C000934501209047012A94209221
:10679000470103E10219102EE8E3F5E04424409498
:1067A00004C0222420925A0208950AE000935B025A
:1067B00000914501222009F400270093450122247D
:1067C000E10DF21D008040FCC895002D1FEF17B9A8
:1067D00018B90E9434310E94343108B90E94343112
:1067E0002E980E9434312E9A0895F8942FEF10338A
:1067F00028F42FEF28B9222727B904C028B927B9D0
:10680000000008B900913101012B0BB90000000014
:10681000000029980E9434310E94343106B1299A2F
:1068200008950F931F93F894009138010F77009308
:10683000380110E40E94F5331F910F910E94F53347
:106840000091380100680093380110E40E94F5338C
:10685000789408950F932F93F89400913801022BA8
:1068600010E40E94F5332F910F9108B90E94343142
:106870000E943431289A0E9434310E943431289881
:106880000E9434310E943431089508B90E94343195
:106890000E943431289AAA27B2E0129711F01B996E
:1068A000FCCF2898AA27B2E0129711F01B9BFCCFCF
:1068B0000E9434310E9434310895289AAA27B2E008
:1068C000129711F01B99FCCF06B12898AA27B2E0C5
:1068D000129711F01B9BFCCF0E9434310E9434317F
:1068E00008950F931F932F93F89400913801022B72
:1068F00010E40E94F5332F911F910F91009508B974
:106900001F9310952C9814FD2C9A2D9815FD2D9AF7
:106910001F9112951095107F00913101012B0BB939
:106920000E9434310E943431289A0E9434310E94EE
:10693000343128980895002E041B002D012E150BCC
:10694000102D022E260B202D032E370B302D0895EF
:1069500015911D930A95E1F7089503E100939F06B1
:1069600008E80093A0060895B4E0A0EB11234AF4D0
:10697000B4E0ADEE2091B00406E0029FA00DB11D81
:106980001095A10F10E0B11F0C910895112329F06B
:10699000B4E0A0EB012E112406C0B4E0ADEE1091DE
:1069A000B00406E0019FA00DB11D0D910895B4E063
:1069B000ADEE0091B00416E0109FA00DB11D14962D
:1069C0000D911C91089510E00091CE04087009F01B
:1069D00011E00E94C6340E70089500E20093A701F2
:1069E0000093A8010093A9010093AA010093AB01B1
:1069F0000093AC010093AD010093AE010093AF0191
:106A00000093B001F89405E10093C80178940895CB
:106A100000E200938F010093900100939101009395
:106A200092010093930100939401009395010093C8
:106A300096010093970100939801F89405E1009363
:106A4000C60178940895E0EEF5E00091B104069552
:106A5000077018E0109FE00DF11D05910093A7014C
:106A600005910093A80105910093A9010591009358
:106A7000AA0105910093AB0105910093AC0105912A
:106A80000093AD0105910093AE0100E20093AF01C8
:106A90000093B00105E10093C8010895B1E0A2EEB2
:106AA0000091D104102F0F7705351CF0107810934A
:106AB000D10416E0019FA00DB11D0E943731302F87
:106AC00031700093910611960E943731202F209348
:106AD000920611960E943731102F1093930611964B
:106AE0000E943731009394060F9311960E9437311C
:106AF0000093950611960E943731009396060F91E8
:106B0000089545E00E944F2E0091AB02002309F04A
:106B100008950DE400937C030AE300937F03009142
:106B2000B201009380030091B301009381030091AF
:106B3000B401009382030091B50100938303009197
:106B4000B601009384030091B7010093850300917F
:106B5000B801009386030091B9010093870300E216
:106B60000093880348E03327222711270091D1049E
:106B70000E944F2E0091B80100937D030093E9031A
:106B80000091B90100937E030093EA03E0EEF5E083
:106B9000009191060E70069518E0109FE00DF11D12
:106BA000059100938903059100938A030591009351
:106BB0008B03059100938C03059100938D03059140
:106BC00000938E03059100938F030591009390032A
:106BD00000E20093AB0208950091AB06002309F494
:106BE00008950091FD06002309F00895F7E0E6E519
:106BF000B6E0ADEA28E61D911F7D05910117C1F4AD
:106C00000093FF061C911F7D04910117A9F40093C6
:106C10000007119611270C910B3309F41FEF109305
:106C20005F023196C591D491FE01D7E0C1E009948D
:106C300033962A9511F704C0119733962A95D9F601
:106C4000D6E0CFEF0FE309930FEF00935F0202E06E
:106C500011C03327222711275FEF48E00E944F2EF3
:106C60000091B70109930091B80109930091B9010E
:106C7000099306E01BE318830093FE060093FD06CC
:106C80000091C10000620093C10000270093AB0691
:106C900000915F0200FF0E94AD340895112371F04E
:106CA00010E30091320105FD11E31993199310E3EC
:106CB0000091170407FD11E319931AC00D91099370
:106CC0000E948A4302300AF0BBCF302F0E948A43D1
:106CD00002300AF0B5CF10913201332329F415FDAB
:106CE0001F7D1093330104C015FF10621093330110
:106CF00006E0C0CF112341F000916B0240916D027C
:106D000040FD00916C02A5CF63E00E9453430AF45A
:106D100097CF222309F094CF10936C020FEF0093CA
:106D20006D0206E0A7CF112341F000916F02409160
:106D3000710240FD009170028CCF63E00E945343CA
:106D40000AF47ECF222309F07BCF109370020FEF5D
:106D50000093710206E08ECF112349F010E30091F9
:106D6000E004007409F011E3199304E083CF0E945A
:106D70008A4302300AF064CFF8941091E0041F7B3C
:106D8000012B0093E004789404E074CF112369F0A0
:106D90000E94E33413960C910870069506950695AB
:106DA0000395005D099304E065CF0E948A4301309A
:106DB00019F0023009F044CF0A95000F000F000FC0
:106DC0000F93F8940E94E33413960C91077F1F9160
:106DD000012B0C9378940FEF0093270204E04ACF25
:106DE000112361F00E94D73400710695069506952F
:106DF00006950395005D099304E03CCF0E948A4309
:106E0000013019F0023009F01BCF0A95000F000F76
:106E1000000F000F0F93F8940E94D7340E910F7E4D
:106E20001F91012B0C9378940FEF0093270204E03D
:106E300021CF112349F010E30091CE04017009F035
:106E400011E3199304E016CF0E948A4302300AF03E
:106E5000F7CEF8941091CE041E7F012B0093CE0440
:106E6000789404E007CF112349F010E300913B012F
:106E7000007809F011E3199304E0FCCE0E948A43E4
:106E800002300AF0DDCEF8940F930E94D7340F7DC4
:106E90001F91110F110F110F110F110F012B0E93D5
:106EA000789404E0E7CE112339F00091D70410E381
:106EB000010F099304E0DECE0E948A4308300AF0F5
:106EC000BFCEF8940093D704789404E0D3CE112376
:106ED00019F00091E204BDCE63E00E9453430AF42E
:106EE000AFCE222309F0ACCE1093E20406E0C2CE6E
:106EF000112349F010E30091E004007109F011E35F
:106F0000199304E0B7CE0E948A4302300AF098CE6B
:106F1000F8941091E0041F7E002311F000E1102B83
:106F20001093E004789404E0A5CE00271123A9F083
:106F30000091DC048ECE01E0112379F00091DC0495
:106F400088CE02E0112349F00091DC0482CE03E0F8
:106F5000112319F00091DD047CCE0F9363E00E94B1
:106F600053430F910AF46CCE222309F069CE202FEF
:106F700006E0222319F41093DC047CCE213019F4AE
:106F80001093DC0477CE223019F41093DC0472CE17
:106F90001093DD046FCE112319F00091E40459CE53
:106FA00063E00E9453430AF44BCE222309F048CEFB
:106FB0001093E40406E05ECE112319F00091E3047F
:106FC00048CE63E00E9453430AF43ACE222309F0EC
:106FD00037CE1093E30406E04DCE112319F0009153
:106FE000DB0437CE63E00E9453430AF429CE222308
:106FF00009F026CE1093DB0406E03CCE112349F0C5
:1070000010E30091E004007209F011E3199304E029
:1070100031CE0E948A4302300AF012CEF8941091C9
:10702000E0041F7D002309F010621093E0047894BF
:1070300004E020CE112319F00091E5040ACE63E0AC
:107040000E9453430AF4FCCD222309F0F9CD10939A
:10705000E50406E00FCE0091E80300680093E80322
:1070600003E008CE112319F00091CC04F2CD63E0C7
:107070000E9453430AF4E4CD222309F0E1CD10939A
:10708000CC0406E0F7CD112349F010E30091DF04B2
:10709000007409F011E3199304E0ECCD0E948A43D7
:1070A00002300AF0CDCDF8941127002309F010E446
:1070B0001093DF04789404E0DDCD112339F010E360
:1070C0000091E604010F099304E0D4CD0E948A43A5
:1070D00003300AF0B5CDF8940093E604789404E008
:1070E000C9CD112349F010E30091E004007809F0C4
:1070F00011E3199304E0BECD0E948A4302300AF0E6
:107100009FCDF8941091E0041F77002309F01068D8
:107110001093E004789404E0ADCD0091E8030160A1
:107120000093E80303E0A6CD112321F010E00E94B4
:107130008E43A0CD10E00E94B7430AF481CD9ACDD2
:10714000112321F011E00E948E4394CD11E00E94A2
:10715000B7430AF475CD8ECD112349F010E30091A9
:10716000CF04087009F011E3199304E083CD0E9465
:107170008A4302300AF064CDF8941091CF04177F4F
:10718000002309F018601093CF04789404E072CDC6
:1071900000913208402F10913308412B2091340880
:1071A000422B30913508432B31F445E335E320E39E
:1071B00010E300E30EC0552748E00E944F2E409197
:1071C000B5013091B6012091B7011091B80100913D
:1071D000B9014993399329931993099308E04ACD4A
:1071E000112391F00091D8040F773327222711271C
:1071F0005FEF48E00E944F2E0091B8010993009183
:10720000B901099305E036CD62E00E9453430AF4C8
:1072100017CD222309F014CD15310AF011CDF894C1
:107220000091D8040078102B1093D804789405E0CE
:1072300021CD112339F00091BE0410E3010F099311
:1072400004E018CD0E948A4302300AF0F9CC009382
:10725000BE0404E00FCD112321F024E0F4E0E3ECC0
:107260000FC00C91005302300AF0EACCF4E0E3ECDA
:10727000442734E019C0112379F024E0F4E0EFEB67
:10728000019110E30A3012F011E60A50010F099340
:107290002A95B1F707E0EECC0C91003309F0D0CC81
:1072A000F4E0EFEB4FEF34E00E948A43442389F48B
:1072B0000A308AF0102F10620AE0113361F0039552
:1072C000123349F00395133331F00395143319F059
:1072D000B7CC0930EAF701933A9531F707E0CACC09
:1072E000112321F000E3099304E0C4CC0E948A43F7
:1072F00010E3002351F0013019F0023021F0A0CC4E
:107300000E94ED4302C00E9419440091CE04077F01
:107310000093CE0404E0AECC112349F000E31091B9
:10732000CE04187009F001E3099304E0A3CC0E9495
:107330008A4310E3002351F0013009F081CC009121
:10734000CE0408600093CE0404E094CC0091CE04F7
:10735000077F0093CE0404E08DCC112349F010E3A5
:1073600000913A01027009F011E3199304E082CC14
:107370000E948A4302300AF063CCF89410913401E1
:107380001D7F000F00950270012B0093350178944A
:1073900004E070CC00910E04002309F04AC01123D0
:1073A00021F110E00E94C634007340911004443073
:1073B0005CF04C304CF410E31993199319930023AB
:1073C00009F411E3199374C0003224F031F010E392
:1073D00024E305C012E324E302C011E328E3199378
:1073E000299310E31993199363C064E00E945343F7
:1073F0000AF426CC4091100444305CF04C304CF43C
:1074000012300CF01DCC109511701295212F3FEC0D
:1074100044C038EE43E01317240700E338F030EDA2
:1074200047E01317240700E208F000E1202F3FECAB
:1074300034C01123A9F010E00E94C63410E307FD08
:1074400011E3199310E306FD11E3199310E305FD11
:1074500011E3199310E304FD11E3199307E00ACC3B
:107460000E948A4302300CF0EBCB202F220F0E94A7
:107470008A4302300CF0E4CB202B220F0E948A4377
:1074800002300CF0DDCB202B220F0E948A43023009
:107490000CF0D6CB202B22953FE010E00E94C634A2
:1074A0000323022B0E930FEF009351030093E1038C
:1074B00007E0E0CB112369F010E00E94C634007CA5
:1074C000029506950695039510E3010F099304E0D4
:1074D000D1CB0E948A43002311F005300CF0B0CBD1
:1074E0000A95000F000F0295202F10E00E94C6346D
:1074F0000F73022B0E930FEF009351030093E103E0
:1075000004E0B8CB112359F010E00E94C634007398
:107510000295039510E3010F099304E0ABCB0E94A1
:107520008A43002311F005300CF08ACB0A950295AE
:10753000202F10E00E94C6340F7C022B0E930FEF19
:10754000009351030093E10304E094CB112359F01D
:1075500000E3099309930E94D734107612951063C3
:10756000199306E087CB0E948A430E948A430E94B7
:107570008A43002339F0023029F0043019F0063034
:1075800009F05ECB02950F930E94D7341F790F91BB
:10759000012B0C930FEF0093270206E06BCB112316
:1075A00049F010E30091E704002309F011E3199377
:1075B00004E060CB0E948A4302300AF041CBF89489
:1075C0000093E704789404E055CB07E3099301E3C3
:1075D000099300E3099306E04DCB10E00E948E432F
:1075E00000910E040023E1F00091BC041091BB0453
:1075F0002091BA043091B9045FEF48E00E944F2E09
:107600000091B10109930091B60109930091B7016E
:1076100009930091B80109930091B901099306C03B
:1076200000E2099309930993099309930091B8041F
:107630001091B7042091B6043091B5045FEF48E093
:107640000E944F2E0091B10109930091B601099358
:107650000091B70109930091B80109930091B90114
:10766000099310E30091BD0407FD11E3199310E3A2
:107670000091BD0400FD11E3199310E219930091EC
:10768000E903006309930091EA030063099310E39F
:107690000091340106FD11E319930E9432451993BC
:1076A00010E30091040400FD12E3199310E300912C
:1076B000030400FD11E3199310E30091CE0403FDD0
:1076C00011E3199300E309930993099300E20993E5
:1076D00006E2D0CA112341F13091D9032091DA0397
:1076E0001091DB030091DC0340910E04442341F030
:1076F0003091DD032091DE031091DF030091E00360
:107700005FEF48E00E944F2E0091B1010993009174
:10771000B60109930091B70109930091B80109934B
:107720000091B90109933DC00D91003229F00B324F
:1077300019F00D3209F084CA09930F9364E00E9496
:10774000534312F40F917CCA012F122F083E43E0DD
:10775000140718F431E022E30FC0003D47E014079E
:1077600018F432E024E608C0083843E1140710F0AA
:107770000F9166CA33E02AEF306830935602332700
:107780000E946F441F911D3209F4019510910E045F
:1077900010FF0093540210FD009355020FEF009369
:1077A000E10308E067CA112361F010E30091CF0400
:1077B00000730695069506950695010F099304E05A
:1077C00059CA0E948A4303300AF03ACAF894000F5B
:1077D000000F000F000F1091CF041F7C102B10938F
:1077E000CF04789404E046CA112349F000911A01AD
:1077F00010918002112311F000917F022ACA63E0E8
:107800000E9453430AF41CCA222309F019CA1034F7
:107810000AF016CA15300AF413CA10937F020FEF4C
:107820000093800206E026CA112349F010E300917C
:107830003401067009F011E3199304E01BCA0D919D
:107840000993F7E0EFE41CE022270D9109930C3334
:1078500009F42FEF01931A95C1F734961CE00D91AE
:10786000099301931A95D9F701E0222309F400E85E
:107870000093F1030FEF0093ED030CE1FBC911231B
:1078800041F010E30091CF040770010F099304E069
:10789000F1C90E948A4305300AF0D2C9F8941091C8
:1078A000CF04187F102B1093CF04789404E0E2C922
:1078B000112339F010E30091AC0200FD11E319939C
:1078C00010C00E948A431127002321F01FEF0130CE
:1078D00009F0B6C91093AC02109510FF13951093E0
:1078E000930304E0C7C9112341F010E30091E004C1
:1078F0000370010F099304E0BDC90E948A4304305C
:107900000AF09EC9F8941091E0041C7F102B10938C
:10791000E004789404E0AEC9112349F010E300912B
:10792000EA04002309F011E3199304E0A3C90E94BB
:107930008A4302300AF084C9F89488940795079521
:107940000093EA04789404E095C9112351F000E211
:1079500009930091E903006309930091EA030993F5
:1079600019C00D9109930D910F930C910F931197DD
:1079700062E00E9453430AF402C015351CF00F91D7
:107980000F9108C00F910093EA030F910093E90350
:107990001093D10406E06EC9112321F00E943245F4
:1079A00019932DC00C91099322270333B1F023952D
:1079B000073399F02395023381F02395013369F061
:1079C0002395053351F02395043339F0239506337D
:1079D00021F02395093309F033C9220F10E00E94EA
:1079E000C634017F022B0E930E7000931004109189
:1079F000CE0413FF009311040FEF0093270204E05D
:107A000039C9112341F0009172021091750210FDE5
:107A1000009174021EC963E00E9453430AF410C926
:107A2000222309F00DC9109374020FEF0093750221
:107A300006E020C90D9109930D91099362E00E941F
:107A4000534315350AF0FCC8B1E0A2EE06E0019FF1
:107A5000A00DB11D0E9437310F700F9301700F936D
:107A600011960E9437310F9311960E9437310F9370
:107A700011960E9437311F912F913F915FEF48E09F
:107A80000E944F2E00E30993099309930091B201DC
:107A900009930091B30109930091B40109930091F6
:107AA000B50109930091B60109930091B7010993BB
:107AB0000091B80109930091B90109930F910695BE
:107AC0000E943645199300E309930993099309939A
:107AD00000E2099308E1CEC80D9109930D91099335
:107AE00062E00E94534315350AF0AAC81F9368E06C
:107AF0000E9453435F910AF4A3C80C9100530AF407
:107B00009FC80A300AF09CC809930E944D45660F31
:107B1000B1E0A2EE06E0059FA00DB11D042F01709B
:107B2000062B0E943E311196032F0E943E31119682
:107B3000022F0E943E311196012F0E943E3100E338
:107B4000099309930993099308E194C8112339F023
:107B50000E94D73420E314FD21E3299311C00E9431
:107B60008A433327002321F030E1013009F068C84F
:107B70000E94D7341F7E132B1C930FEF0093270214
:107B800004E078C8112341F0009160021091630273
:107B900010FD009162025DC863E00E9453430AF445
:107BA0004FC8222309F04CC8109362020FEF0093D4
:107BB000630206E05FC8112371F00E94D7341C7085
:107BC000012F10E3002321F011E3043009F012E348
:107BD000199304E04FC80E948A4303300AF030C86A
:107BE000F8940F930E94D734137F0F91000F000F6A
:107BF000102B1C93789404E03DC8112379F020E306
:107C0000009132010370002320E331F0023021F0B3
:107C100021E3013009F022E3299319C02C91299323
:107C20003091320130FD3D7F3270203341F031E040
:107C3000213329F033E0223311F00C942036F894EC
:107C4000009133010C7F032B00933301789404E0FF
:107C500011C8112309F11127009164022091CE046B
:107C60002670243031F0263021F033272AE00E949C
:107C70006F443327222711275FEF48E00E944F2EE1
:107C80000091B70109930091B80109930091B901DE
:107C9000099306E00C943A3663E00E94534312F4D1
:107CA0000C9420364091CE044670443051F046305A
:107CB00041F01C3010F00C9420360AE0019F102D8A
:107CC00004C0113810F00C942036109367020FEFA7
:107CD0000093680206E00C943A36112359F010E341
:107CE0000091E0040C7006950695010F099304E0DD
:107CF0000C943A360E948A43043012F00C942036D9
:107D0000F8941091E004137F000F000F102B1093D4
:107D1000E004789404E00C943A36112349F0009181
:107D20007A0210917D0210FD00917C020C9429369C
:107D300063E00E94534312F40C942036222311F086
:107D40000C94203610937C020FEF00937D0206E026
:107D50000C943A36112351F010E30091D8040078C6
:107D600009F011E3199304E00C943A360E948A4317
:107D7000023012F00C942036F8941091D8041F773A
:107D8000002309F010681093D804789404E00C9450
:107D90003A36112379F010E300910F042091110479
:107DA000243024F400FD11E3199314C007FD11E3FE
:107DB000199310C00E948A43023012F00C942036AE
:107DC000112700FD10E1009132010F7E012B00937D
:107DD0003301789404E00C943A36112339F010E31F
:107DE0000091F30307FD11E319930DC00E948A432C
:107DF000023014F00C942036F89406950795016033
:107E00000093F303789404E00C943A36112331F193
:107E100033270091820210918302112381F4109183
:107E2000170100911801055C104032F400E309933A
:107E3000099305E00C943A3621E40E946F4422270E
:107E400011275FEF48E00E944F2E0091B80109937F
:107E50000091B901099305E00C943A3662E00E9462
:107E6000534312F40C9420361D3010F00C9420363D
:107E7000109382020FEF0093830205E00C943A36D0
:107E8000112351F010E30091CE0406700695010F06
:107E9000099304E00C943A360E948A43043012F0AD
:107EA0000C942036F8941091CE04197F000F102BFB
:107EB0001093CE04789404E00C943A36112361F0C8
:107EC00020E300913201037019F000FD01C021E3AD
:107ED00010E3199329931BC00E948A43023014F0C7
:107EE0000C9420360E948A4332E0013041F0009128
:107EF000320100FD0CC001FF0AC0332700C0F89416
:107F0000009133010C7F032B00933301789405E03B
:107F10000C943A3644275527662777271BC0709163
:107F2000B5046091B6045091B7044091B8044A502A
:107F30005040604070400EC07091B5046091B6042E
:107F40005091B7044091B8048AE0480F80E0581F70
:107F5000681F781F7093B5046093B6045093B704FC
:107F60004093B80403E00C943A36F5E1E9E9059151
:107F70000993059109930591099305910993059139
:107F8000099305910993059109930AE00C943A36F7
:107F9000112349F0009177024091790240FD009150
:107FA00078020C94293663E00E94534312F40C9437
:107FB0002036222311F00C942036109378020FEF14
:107FC0000093790206E00C943A360091E9040370BC
:107FD00011E4010F09930EE2099300E30993009164
:107FE000E904069506950395037010E3010F0993C4
:107FF0000EE209930091E90406950695069506950B
:108000000F7010E30A3012F011E30A50199310E3D5
:10801000010F09930AE00C943A361123C9F100913B
:1080200012040993109169030133F1F010916D036B
:108030000233D1F010916C030333B1F010916E0351
:10804000043391F010917003053371F010916F03B8
:10805000063351F010916A03073331F010916B032E
:10806000083311F00C94203622275FEF48E00E947D
:108070004F2E0091B60109930091B7010993009129
:10808000B80109930091B901099308E00C943A36BC
:108090000E948A4312F0093014F00C9420360063D9
:1080A0000093120404E00C943A360FEF0093DA04C4
:1080B00003E00C943A36112339F010E30091BD042B
:1080C00007FD11E3199318C00E948A4312F0023091
:1080D00014F00C9420361091BD04002319F417FFFE
:1080E00059F002C017FD41F4F8941091340108E0F2
:1080F000102710933501789404E00C943A36F894E4
:1081000000913801086010E40E94F53306ED0E94EA
:10811000453400270E944534789403E00C943A36A5
:10812000112351F020E30E94D734007409F021E3B9
:10813000299304E00C943A360E948A43023012F0EC
:108140000C942036F894202F0E94D7340F7B2223E2
:1081500009F000640E93789404E00C943A36F89495
:1081600000913801086010E40E94F53306ED0E948A
:1081700045340FEF109111041A3019F014300CF03F
:1081800000E80E944534789403E00C943A361123B9
:1081900039F410E30091030400FD11E318830BC0D0
:1081A0000E948A43023012F00C942036112700FD01
:1081B0001FEF1093030404E00C943A36112341F0AE
:1081C00010E30091D504010F099304E00C943A36B2
:1081D0000E948A43083012F00C942036F8940093E1
:1081E000D504789404E00C943A36112381F03327B7
:1081F000222711270091D4045FEF48E00E944F2E00
:108200000091B80109930091B90109930CC062E093
:108210000E94534312F40C942036153514F00C943C
:1082200020361093D40405E00C943A36112381F0E3
:108230003327222711270091D3045FEF48E00E94E3
:108240004F2E0091B80109930091B90109930CC018
:1082500062E00E94534312F40C942036153514F05A
:108260000C9420361093D30405E00C943A36112375
:1082700041F010E30091D604010F099304E00C943F
:108280003A360E948A43053012F00C942036F89456
:108290000093D604789404E00C943A36112341F00C
:1082A00010E30091D204010F099304E00C943A36D4
:1082B0000E948A43053012F00C942036F894009303
:1082C000D204789404E00C943A361123C1F0332799
:1082D0002227009190021AE0019F80015FEF48E0A1
:1082E0000E944F2E0091B60109930091B7010993A6
:1082F0000091B80109930091B901099314C064E099
:108300000E94534312F40C942036012F122F29E0BF
:10831000073F120710F00C94203633272AE00E9402
:108320006F440093CB0407E00C943A36112339F0E4
:1083300010E300910E0400FD11E319930BC00E949D
:108340008A43023012F00C942036112700FD1FEFF3
:1083500010930E0404E00C943A3633272BE110916D
:10836000AE040091AF040E946F4422275FEF48E003
:108370000E944F2E0091B60109930091B701099315
:108380000091B80109930091B901099307E00C9499
:108390003A36112349F0009161024091630240FD99
:1083A000009162020C94293663E00E94534312F458
:1083B0000C942036222311F00C9420361093620284
:1083C0000FEF0093630206E00C943A3610E300913D
:1083D000D90401FD11E319933327222710911B01C2
:1083E00000911C015FEF48E00E944F2E0091B60102
:1083F00009930091B70109930091B8010993009185
:10840000B901099308E00C943A360E948A4302307D
:1084100012F00C9420361091D9041B7F000F000F2E
:10842000102B1093D90404E00C943A3633272227FA
:1084300010911D0100911E015FEF48E00E944F2E38
:108440000091B60109930091B70109930091B80119
:1084500009930091B901099307E00C943A360E9400
:108460008A43023012F00C9420361091D9041E7FFA
:10847000102B1093D90404E00C943A36112329F000
:108480000091CD0403950C94293663E00E94534378
:1084900012F40C942036222311F00C942036113063
:1084A00024F41E3114F00C9420361A951093CD0448
:1084B00006E00C943A36112321F00091C9040C9483
:1084C000293663E00E94534312F40C942036222391
:1084D00011F00C942036112311F40C9420361093D3
:1084E000C90406E00C943A361123C1F03327222741
:1084F0001AE000918F02019F80015FEF48E00E9427
:108500004F2E0091B60109930091B7010993009194
:10851000B80109930091B901099314C064E00E9465
:10852000534312F40C942036012F122F29E0073FF9
:10853000120710F00C94203633272AE00E946F4473
:108540000093CA0407E00C943A36112321F00091FD
:108550008C020C94293663E00E945343222312F4C8
:108560000C9420361093C70406E00C943A3611237D
:1085700071F010E30091D004002339F011E30230D0
:1085800021F012E3013009F013E3199319C00E949E
:108590008A43043012F00C9420361127002359F03E
:1085A00012E0013041F011E0023029F013E0033015
:1085B00011F00C9420361093D0040FEF0093270293
:1085C00004E00C943A36112339F010E30091BD0415
:1085D00000FD11E3199318C00E948A4312F0023083
:1085E00014F00C9420361091BD04002319F410FFF0
:1085F00059F002C010FD41F4F8941091340104E0E8
:10860000102710933501789404E00C943A36002733
:108610001127222733271BC03091B9042091BA04B7
:108620001091BB040091BC040A501040204030401F
:108630000EC03091B9042091BA041091BB0400918E
:10864000BC048AE0080F80E0181F281F381F3093F1
:10865000B9042093BA041093BB040093BC0403E054
:108660000C943A36112381F03327222711270091E9
:10867000E1045FEF48E00E944F2E0091B80109939A
:108680000091B90109930CC062E00E94534312F4B7
:108690000C942036173114F00C9420361093E1041A
:1086A00005E00C943A361127222733274427552713
:1086B0000D9109930E9481430AF1100F251F351F68
:1086C000451F6A95C9F0110F221F331F441F4F9396
:1086D0003F932F931F93110F221F331F441F110F1E
:1086E000221F331F441F0F91100F0F91201F0F9156
:1086F000301F0F91401FDCCF002708950FEF00239C
:108700000895005320F00A3010F4002308950FEF6D
:10871000002308950D910993005308950E94C634D3
:10872000302F31702D911D910C915FEF48E00E9428
:108730004F2E00E30993099309930091B201099325
:108740000091B30109930091B40109930091B5011F
:1087500009930091B60109930091B7010993009123
:10876000B80109930091B90109930EE00895712FA2
:108770000D9109930E9481430AF42CC00D91099335
:108780000E9481430AF426C00D9109930E948143FF
:108790000AF420C068E00E9453430AF41BC00C9105
:1087A0000B3309F017C04F933F932F931F93F89407
:1087B000172F0E94C63411970E7F1F912F913F9162
:1087C0004F91402B4D933D932D931C9378940EE045
:1087D000002308950FEF0023089510E00E94C6348F
:1087E000402F4E701091CE0413FD409311041D9143
:1087F0002D913C91AF93BF930F931F932F933F9372
:1088000011E00E94C634402F4E70409310041D9119
:108810002D913C914F914C934F914E934F914E938C
:108820004F914E93BF91AF913C932E931E930E9315
:108830000895F89410E00E94C634009191060E93BA
:108840000E70009310041091CE0413FF00931104D6
:108850001196009192060D93009193060D9300914D
:1088600094060D93009195060D930091960600686D
:108870000C930FEF009327020093E103002700936E
:108880005402009355020E94AD3478940895A801D3
:108890005A014FE35527BA019A0185010E946F449E
:1088A000A8011A01260E371E36942794B1019101B2
:1088B00085010E946F44A8011A01260E371E3694C6
:1088C0002794B101910185010E946F44A8011A010A
:1088D000260E371E36942794B10181010895EE24A7
:1088E000DD2480E1000F111FEE1CDD1CE216D30613
:1088F00018F0E21AD30A03958A95A1F70895029F0A
:10890000C001129F900D039F900D8C0108959091CE
:10891000CF0497708827F9E1E4E35AE0589FD0012B
:108920005527A90FB51FEA0FFB1F359654919517D0
:1089300009F04CC0D0011496F9E1E4E3EA0FFB1F03
:1089400054915E33B1F5F9E1E4E3E00DF11D759169
:108950006591559145910E949B34E4F1C1E04C2F03
:10896000480F6AE0649FD0015527A90FB51FF9E1B0
:10897000E4E3EA0FFB1F359654919517B9F4D00143
:108980001496F9E1E4E3EA0FFB1F54915C3371F4B0
:10899000F9E1E4E3E00DF11D759165915591459183
:1089A0000E949B34CCF0C1F08C0F10C0C395C63030
:1089B000B1F65D3359F4F9E1E4E3E00DF11D759191
:1089C0006591559145910E949B3431F08395873292
:1089D0000CF4A1CF68940895E8940895B3E0ACE74F
:1089E00015E100E2F8940D931A95E9F700E200937F
:1089F000AB027894089520533AE0329F1053010E51
:108A00003327E8E0F9E10A95000FE00FF31F059125
:108A10001491000D131F0C5110402227552748E0D8
:108A20000E944F2E2091B7011091B8010091B90119
:108A300008950F7002951127B7E0AFE4A00FB11FA2
:108A4000F8E0E6E11CE022270D910C3309F42FEF4A
:108A5000222309F000E201931A95B1F707E1009390
:108A60000B04089510E00E94C6340E7011E3063026
:108A700099F012E3043081F013E3003069F014E35D
:108A80000A3051F015E3083039F016E30C3021F0CC
:108A900017E3023009F019E3089566E0013399F015
:108AA00064E0023381F060E0033369F06AE004338C
:108AB00051F068E0053339F06CE0063321F062E0F4
:108AC000073309F06EE0089500EC00931704F89462
:108AD0000091420100640F7D10ED0E9411347894E2
:108AE000F89400913B010170006D10E70E94113471
:108AF00000913801086010E40E94F53306ED0E94F1
:108B000045340FEF0E944534789444E68DE0772792
:108B100066275527109144011078062F00950F778E
:108B2000012B0E94744610EF0E941134052F0F771D
:108B3000072B0E94744610EE0E9411340E945E467C
:108B40000AF485C04F935F938F930E9486460E94DC
:108B5000A4460E9408478F915F914F9100910201B6
:108B6000041738F45093A6066093A5067093A706E1
:108B7000402F08170CF472C08894552309F4089408
:108B8000551F57FFC7CF8894662309F40894661FC2
:108B900067FFBFCF772311F470E8BACF03E0800FEF
:108BA00089310CF4B4CF8DE06091A5066695909163
:108BB000A506992311F497E003C0990F97FD9FE74D
:108BC0005091A60656953091A606332311F437E04E
:108BD00003C0330F97FD9FE7109144011078062FD3
:108BE00000950F77012B0E94744610EF0E941134FC
:108BF0007091A706052F0F77072B0E94744610EE81
:108C00000E9411340E945E4612F13F934F935F938E
:108C10008F939F930E9486460E94A4460E94084715
:108C20009F918F915F914F913F91009102010417A5
:108C300028F45093A6066093A506402F081774F0F9
:108C40005395531749F66395691709F0B9CF0FE7A4
:108C50000093A30600270093A40612C00091A50666
:108C60000E94744600950F770093A3060091A60614
:108C70000E9474460F771091A706012B0093A4065B
:108C8000F89400913801086010E40E94F53306ED75
:108C90000E94453400270E94453400913B0110E7B3
:108CA0000E9411340091420110ED0E941134009194
:108CB00017040F7B00931704789408950BE000933A
:108CC00016040091320105FD02C028940895009118
:108CD00016040023B1F7A894089500931604009198
:108CE00016040023E1F70895102F107800FD10649A
:108CF00001FD106202FD106103FD186004FD1460A7
:108D000005FD126006FD1160012F0895F894109181
:108D1000A0040091A10478940E94EE4630936B0366
:108D20000093060110930501309123012091240145
:108D30000217130740F0020F131F169507951093A3
:108D40002301009324010895F8941091A204009146
:108D5000A30478940E94EE4630936A0310930301B3
:108D600000930401F8943091A4023323A9F133272E
:108D70003093A40232E03093A30278943091210121
:108D80002091220102171307EAF44091A0025091AA
:108D9000A102451709F14093A10289013695279553
:108DA00036952795369527953695279536952795A7
:108DB000422F432B09F421E0021B130B4AF4002736
:108DC000112706C0F8943BE43093A0023093A1022F
:108DD0001093210100932201789408951695079528
:108DE00016950795009F112D2EE2129E110E1F92CF
:108DF00029E8129F80012091CE042670243031F0A2
:108E0000263021F02AE033270E946F443F910895D5
:108E10007894112700916A0310932601009327018B
:108E2000000F111F000F111F000F111F000F111F46
:108E3000000F111F000F111F0E9447441F930F9333
:108E4000112700916B031093280100932901000F53
:108E5000111F000F111F000F111F000F111F000F16
:108E6000111F000F111F0E944744309126012091CD
:108E700027010E947F44000F111F2F913F910E94F4
:108E80006F443091260120912701020F131F30916A
:108E9000280120912901A901020F131F2AE033277D
:108EA0000E947F443091260120912701241B350B1D
:108EB0001AF00901102811F4332721E00E946F44B1
:108EC0000F931F931AE0019FF894009202011092F1
:108ED000010178941F910F910A50104010F400275F
:108EE0001127102F002728E233270E946F4410918A
:108EF000340116FF0027009369030895B1E0A0E054
:108F0000F8E0E2E7F8940C9111270E94A547B1F42C
:108F10001FEF0E94A54791F41AEA0E94A54771F439
:108F200015E50E94A54751F40C931196AE17BF07A3
:108F300049F778940AE100935C0208950C937894C1
:108F40000AE1019500935C0208951C932C9112177D
:108F500008953091FD063323E1F7D6E0CFEF30E2FC
:108F600039933327222711275FEF48E00E944F2EC5
:108F70000091B70109930091B80109930091B901DB
:108F8000099305E00E943A36089559980E943431B9
:108F90000E9434310E9434310E9434310E943431B5
:048FA000599A08953D
:00000001FF
